:020000040000FA
:10000000DBEF3CF0F76A140FF66E000EF7220900E2
:10001000F55012000A4E494320696E6974206572DA
:1000200072200000F76A340FF66E000EF722090006
:10003000F5501200204E494320706B742065727297
:100040002000F76A520FF66E000EF7220900F550F5
:100050001200204E49432070747220657272200095
:10006000F76A700FF66E000EF7220900F5501200C5
:100070004E6F2064617974696D650D0A0000F76A3E
:100080008E0FF66E000EF7220900F55012000D0AD1
:1000900053657269616C206E756D3F200000F76AD0
:1000A000AE0FF66E000EF7220900F550120048540C
:1000B00054502F20323030204F4B0D0A0D0A4E6F16
:1000C00020576562207061676573210D0A00F76A29
:1000D000DE0FF66E000EF7220900F550120063687D
:1000E00065636B656400F76AF60FF66E000EF72223
:1000F0000900F550120070617373776F72642E6897
:10010000746D0000F76A140FF66E010EF7220900F5
:10011000F55012006572726F722E68746D00F76A86
:100120002E0FF66E010EF7220900F550120020285E
:10013000444843502900F76A460FF66E010EF72235
:100140000900F55012002028537461746963290076
:10015000F76A600FF66E010EF7220900F5501200E3
:1001600057656220536D61727420503138413639C1
:1001700039390000F76A840FF66E010EF722090084
:10018000F550120056657220312E30340000F76AA7
:100190009E0FF66E010EF7220900F55012004B5328
:1001A0002D313137464D2D560000F76ABA0FF66EE5
:1001B000010EF7220900F55012004B532D31313555
:1001C000464D2D560000F76AD60FF66E010EF72247
:1001D0000900F55012004B5449204E6574776F7238
:1001E0006B730000F76AF40FF66E010EF722090038
:1001F000F55012000D0A44484350204950207363C3
:10020000616E6E696E670000F76A180FF66E020E77
:10021000F7220900F55012004B533131372D000001
:10022000F76A300FF66E020EF7220900F550120041
:100230004B533131352D0000F76A480FF66E020E30
:10024000F7220900F55012000D0A0D0A0000F76AA6
:100250005E0FF66E020EF7220900F5501200576588
:100260006220536D61727420503138413600F76A54
:100270007E0FF66E020EF7220900F5501200436F52
:100280006E6669672000F76A960FF66E020EF72217
:100290000900F55012000D0A0D0A495020616464EE
:1002A000723A2000F76AB40FF66E020EF7220900C8
:1002B000F55012000D0A4E65746D61736B3A2000A3
:1002C000F76AD00FF66E020EF7220900F550120001
:1002D0000D0A476174657761792049503A20000022
:1002E000F76AF00FF66E020EF7220900F5501200C1
:1002F0000D0A4D616320616464723A200000F76A60
:100300000E0FF66E030EF7220900F55012000D0ACB
:1003100041444D3620436865636B0000F76A2C0F3B
:10032000F66E030EF7220900F5501200204F4B2005
:100330002100F76A420FF66E030EF7220900F5500E
:100340001200204661696C6564202100F76A5C0F29
:10035000F66E030EF7220900F55012000D0A39332C
:1003600043343620436865636B00F76A7A0FF66E94
:10037000030EF7220900F55012000D0A52544C38B2
:1003800030313920436865636B00F76A9A0FF66E67
:10039000030EF7220900F55012000D0A32344C43C7
:1003A00032353620436865636B00010EEA6E640ED9
:1003B000E96EEF50D8B4EAEF01F0060E016E006A64
:1003C000002EFED7012EFBD77B0E006E002EFED72F
:1003D000EF2EF3D7000C01011A51E96E1B51EA6EA2
:1003E00000011FC1EFFF010E01011A25E96E000E89
:1003F0001B21EA6E00011EC1EFFF020E01011A254A
:10040000E96E000E1B21EA6E00011DC1EFFF030E15
:1004100001011A25E96E000E1B21EA6E00011CC1C4
:10042000EFFF000C0101636B626B0001010162517F
:100430000508D8B003D000012DEF02F0000162C121
:10044000A9FFA69CA69EA680A850010163270001D3
:100450000101622B000116EF02F00101631F6351DD
:10046000016E0001000CA96A36C0A8FFA69CA69EDA
:10047000A684F250006EF29E0F01550EA76EAA0ED2
:10048000A76EA6820001A6B243EF02F0A694005028
:10049000F212010EA96E37C0A8FFA69CA69EA684E4
:1004A000F250006EF29E0F01550EA76EAA0EA76EB7
:1004B000A6820001A6B25AEF02F0A6940050F212F2
:1004C000020EA96E1CC0A8FFA69CA69EA684F25090
:1004D000006EF29E0F01550EA76EAA0EA76EA682A1
:1004E0000001A6B271EF02F0A6940050F212030EC2
:1004F000A96E1BC0A8FFA69CA69EA684F250006E03
:10050000F29E0F01550EA76EAA0EA76EA6820001DD
:10051000A6B288EF02F0A6940050F212040EA96E63
:100520001AC0A8FFA69CA69EA684F250006EF29E5A
:100530000F01550EA76EAA0EA76EA6820001A6B2E5
:100540009FEF02F0A6940050F212050EA96E19C09A
:10055000A8FFA69CA69EA684F250006EF29E0F01F4
:10056000550EA76EAA0EA76EA6820001A6B2B6EF20
:1005700002F0A6940050F212130EA96E24C0A8FF38
:10058000A69CA69EA684F250006EF29E0F01550E08
:10059000A76EAA0EA76EA6820001A6B2CDEF02F04A
:1005A000A6940050F212140EA96E23C0A8FFA69CB8
:1005B000A69EA684F250006EF29E0F01550EA76E05
:1005C000AA0EA76EA6820001A6B2E4EF02F0A694DE
:1005D0000050F212150EA96E22C0A8FFA69CA69E7E
:1005E000A684F250006EF29E0F01550EA76EAA0E61
:1005F000A76EA6820001A6B2FBEF02F0A6940050FF
:10060000F212160EA96E21C0A8FFA69CA69EA68473
:10061000F250006EF29E0F01550EA76EAA0EA76E45
:10062000A6820001A6B212EF03F0A6940050F212C7
:10063000170EA96E28C0A8FFA69CA69EA684F250FD
:10064000006EF29E0F01550EA76EAA0EA76EA6822F
:100650000001A6B229EF03F0A6940050F212180E82
:10066000A96E27C0A8FFA69CA69EA684F250006E85
:10067000F29E0F01550EA76EAA0EA76EA68200016C
:10068000A6B240EF03F0A6940050F212190EA96E24
:1006900026C0A8FFA69CA69EA684F250006EF29EDD
:1006A0000F01550EA76EAA0EA76EA6820001A6B274
:1006B00057EF03F0A6940050F2121A0EA96E25C04F
:1006C000A8FFA69CA69EA684F250006EF29E0F0183
:1006D000550EA76EAA0EA76EA6820001A6B26EEFF7
:1006E00003F0A6940050F21212EC02F001C01AF1CD
:1006F000060EA96E1AC1A8FFA69CA69EA684F2505B
:10070000006EF29E0F01550EA76EAA0EA76EA6826E
:100710000001A6B289EF03F0A6940050F212000C7B
:10072000899289948996800E0101566F090E576F40
:10073000010E586F0001010158510408D8B003D0D0
:100740000001AEEF03F00001D89001015637573792
:1007500000010101582B00019BEF03F08986020E76
:100760000101646F0001D5EC01F0010E0101586F29
:100770000001010158510A08D8B003D00001D7EF99
:1007800003F00001D890010156375737D8A003D0A5
:100790000001CFEF03F000018992D0EF03F08982CE
:1007A000898489940101582B0001B9EF03F08992E3
:1007B000020E0101646F0001D5EC01F08996080E6C
:1007C000006E002EFED789848994000C01015E35ED
:1007D0005F6F5F37FC0E5F175D35646F6437FC0E2B
:1007E00064175E39006E00320032030E00160050AE
:1007F0006411606F5C35646F6437FC0E64175D399B
:10080000006E00320032030E001600506411616F5A
:10081000050E626F010E636F00010101635105084F
:10082000D8B003D0000122EF04F00001D8900101FC
:100830005F3760376137623700010101632B0001C8
:100840000DEF04F08986020E0101646F0001D5EC02
:1008500001F08980010E0101636F00010101635104
:100860001908D8B003D000014EEF04F00001D89071
:1008700001015F37603761376237D8A003D00001CC
:1008800046EF04F00001899247EF04F089828984E1
:1008900089940101632B00012EEF04F0899289965F
:1008A000030E006E002EFED789848994030E006E1D
:1008B000002EFED7898689848994000E80B0010EAF
:1008C0000108D8B45BEF04F0020E0101646F00016F
:1008D000D5EC01F08996080E006E002EFED78984B3
:1008E0008994320E0101646F0001D5EC01F0000C17
:1008F000020EA96E56C1A8FFA69CA69EA684F25021
:10090000006EF29E0F01550EA76EAA0EA76EA6826C
:100910000001A6B289EF04F0A6940050F212030E73
:10092000A96E57C1A8FFA69CA69EA684F250006E91
:10093000F29E0F01550EA76EAA0EA76EA6820001A9
:10094000A6B2A0EF04F0A6940050F212040EA96E15
:1009500058C1A8FFA69CA69EA684F250006EF29EE7
:100960000F01550EA76EAA0EA76EA6820001A6B2B1
:10097000B7EF04F0A6940050F212050EA96E59C10B
:10098000A8FFA69CA69EA684F250006EF29E0F01C0
:10099000550EA76EAA0EA76EA6820001A6B2CEEFD4
:1009A00004F0A6940050F21212EC02F001C062F1C1
:1009B000060EA96E62C1A8FFA69CA69EA684F25050
:1009C000006EF29E0F01550EA76EAA0EA76EA682AC
:1009D0000001A6B2E9EF04F0A6940050F212130E43
:1009E000A96E5AC1A8FFA69CA69EA684F250006ECE
:1009F000F29E0F01550EA76EAA0EA76EA6820001E9
:100A0000A6B200EF05F0A6940050F212140EA96EE3
:100A10005BC1A8FFA69CA69EA684F250006EF29E23
:100A20000F01550EA76EAA0EA76EA6820001A6B2F0
:100A300017EF05F0A6940050F212150EA96E5CC1D6
:100A4000A8FFA69CA69EA684F250006EF29E0F01FF
:100A5000550EA76EAA0EA76EA6820001A6B22EEFB3
:100A600005F0A6940050F212160EA96E5DC1A8FF03
:100A7000A69CA69EA684F250006EF29E0F01550E13
:100A8000A76EAA0EA76EA6820001A6B245EF05F0DA
:100A9000A6940050F212170EA96E5EC1A8FFA69C84
:100AA000A69EA684F250006EF29E0F01550EA76E10
:100AB000AA0EA76EA6820001A6B25CEF05F0A6946E
:100AC0000050F212180EA96E5FC1A8FFA69CA69E48
:100AD000A684F250006EF29E0F01550EA76EAA0E6C
:100AE000A76EA6820001A6B273EF05F0A69400508F
:100AF000F212190EA96E60C1A8FFA69CA69EA6843C
:100B0000F250006EF29E0F01550EA76EAA0EA76E50
:100B1000A6820001A6B28AEF05F0A6940050F21258
:100B20001A0EA96E61C1A8FFA69CA69EA684F250CB
:100B3000006EF29E0F01550EA76EAA0EA76EA6823A
:100B40000001A6B2A1EF05F0A6940050F21244EF06
:100B500007F0010E926E90EC03F001015C6B410E08
:100B60005D6F540E5E6F0001E6EC03F0130E0101A1
:100B7000556F0001010155512208D8B003D0000182
:100B8000D2EF05F0000155C15CF1FF0E01015D6F70
:100B9000040E5E6F0001E6EC03F00101552B00012D
:100BA000BAEF05F0140E01015C6FFF0E5D6FFF0ED2
:100BB0005E6F0001E6EC03F0230E0101556F0001AA
:100BC000010155513F08D8B003D00001F6EF05F000
:100BD000000155C15CF101015D6B5E6B0001E6EC4B
:100BE00003F00101552B0001E0EF05F0010E0101BA
:100BF000556F0001010155510908D8B003D000011B
:100C000012EF06F0000155C15CF1840E01015D6F29
:100C10004F0E5E6F0001E6EC03F00101552B000161
:100C2000FAEF05F0030E01015C6F840E5D6F410E5B
:100C30005E6F0001E6EC03F0080E01015C6FC40E6C
:100C40005D6F4D0E5E6F0001E6EC03F00A0E0101D0
:100C50005C6F590E5D6F020E5E6F0001E6EC03F0F3
:100C60000B0E01015C6F800E5D6F5E6B0001E6ECA8
:100C700003F00C0E01015C6FFA0E5D6F500E5E6F9B
:100C80000001E6EC03F00D0E01015C6FFA0E5D6FE2
:100C9000500E5E6F0001E6EC03F00E0E01015C6F7A
:100CA000550E5D6F5E6B0001E6EC03F00F0E010167
:100CB0005C6F550E5D6F5E6B0001E6EC03F0100E8D
:100CC00001015C6F300E5D6F5E6B0001E6EC03F0BE
:100CD000110E01015C6FFF0E5D6F5E6B0001E6ECB3
:100CE00003F0120E01015C6F360E5D6F5E6B00014A
:100CF000E6EC03F02C0E01015C6FD00E5D6F5E6BB5
:100D00000001E6EC03F02D0E01015C6F450E5D6FF6
:100D1000560E5E6F0001E6EC03F00101556B000119
:100D2000010155510708D8B003D00001B9EF06F012
:100D300000010A0E01015525566F000156C1A9FF99
:100D4000A86AA69CA69EA684F250006EF29E0F0191
:100D5000550EA76EAA0EA76EA6820001A6B2AEEF30
:100D600006F0A6940050F2120101552B000190EFFD
:100D700006F00A0EA96E310EA86EA69CA69EA68449
:100D8000F250006EF29E0F01550EA76EAA0EA76ECE
:100D9000A6820001A6B2CAEF06F0A6940050F21295
:100DA0000B0EA96E320EA86EA69CA69EA684F250CB
:100DB000006EF29E0F01550EA76EAA0EA76EA682B8
:100DC0000001A6B2E1EF06F0A6940050F2120C0E5C
:100DD000A96E330EA86EA69CA69EA684F250006E45
:100DE000F29E0F01550EA76EAA0EA76EA6820001F5
:100DF000A6B2F8EF06F0A6940050F212080EA96E03
:100E0000A86AA69CA69EA684F250006EF29E0F01D0
:100E1000550EA76EAA0EA76EA6820001A6B20EEF0F
:100E200007F0A6940050F212090EA96E020EA86EE9
:100E3000A69CA69EA684F250006EF29E0F01550E4F
:100E4000A76EAA0EA76EA6820001A6B225EF07F034
:100E5000A6940050F212C00E0101566FA80E576FF3
:100E6000586B020E596FFF0E5A6FFF0E5B6FFF0E2D
:100E70005C6F5D6BC00E5E6FA80E5F6F606B010EE6
:100E8000616F000178EF04F0000C21C103F0010153
:100E90002051E96E000103C0EAFFECCF03F0ED52F0
:100EA000EF50105C0101246F03501158256F22513F
:100EB0002311D8A403D0000174EF07F00001010151
:100EC0002351255DD8B003D0000185EF07F0000164
:100ED000D8A474EF07F001012251245DD8B003D0EB
:100EE000000185EF07F0000121C103F0010120514D
:100EF000E96E000103C0EAFF11C0ECFFED5210C023
:100F0000EFFF010E016E87EF07F0000E016E000C7F
:100F100074C181FF75C183FF000E956E849200003D
:100F20008482FF0E956E000C0E0E01017127400E9B
:100F30007223070E746F400E756F000188EC07F086
:100F4000080E0101746F000171C175F188EC07F0A2
:100F500072C173F1090E0101746F000173C175F163
:100F600088EC07F0010E6C6E000CFF0E956E71C1DF
:100F700081FF849083CF72F1848001017251016EF0
:100F80000001000C01016F6B000171C070F10101E3
:100F90007053D8B403D00001D1EF07F000012FEF58
:100FA00008F001017051010B7027070E746F400E9D
:100FB000756F000188EC07F00A0E0101746F0001E3
:100FC00070C175F188EC07F00B0E0101746F756B41
:100FD000000188EC07F00101746B120E756F0001BF
:100FE00088EC07F0100E816E000E956E01017051B5
:100FF0007007000AD8A403D0000110EF08F0000128
:1010000001016F516F2B720FE96EEA6AD8B0EA2ABC
:10101000EF50836E8492000084820001F6EF07F0A7
:10102000FF0E956EFF0E0101706F000101017053FC
:10103000D8A403D000012FEF08F00001070E010132
:10104000716F0001B5EC07F00150400B000AD8A405
:101050002FEF08F001017007000116EF08F0000CF7
:101060007152D8B449EF08F06C52D8A446EF08F09A
:1010700071506F5C01016F6F000E7058706F00014E
:1010800070C172F16FC171F194EC07F0C2EC07F01E
:10109000716A6E50705CD8A05AEF08F0D8A456EF71
:1010A00008F06F506D5CD8B05AEF08F070C06EF069
:1010B0006FC06DF0000C29A070EF08F001016F51B6
:1010C0002B266F512B5CD8A003D000016EEF08F0E7
:1010D00000012A2AD8A46EEF08F02B2A80EF08F02E
:1010E00001016F512A266F512A5CD8A003D000015C
:1010F00080EF08F000012B2AD8A480EF08F02A2AFC
:101100002970000C70500408D8B094EF08F0FF0A62
:10111000D8A490EF08F06F50E908D8B094EF08F029
:10112000000E016EADEF08F071501F08D8B09BEFB4
:1011300008F030EC08F07150712A720FE96EEA6A1B
:10114000D8B0EA2A6EC1EFFF6F2AD8B4702A6EC1F8
:101150006FF15BEC08F0010E016E000C29A6C6EFE2
:1011600008F001016D510A08D8B403D00001BFEFA7
:1011700008F000010D0E9EA8BBEF08F0AD6E010156
:101180006D5100019EA8C2EF08F0AD6E29A8CDEF09
:1011900008F06DC16EF182EC08F0000CA96AA69C03
:1011A000A69EA680A850366E010EA96EA69CA69E8D
:1011B000A680A850376E020EA96EA69CA69EA68099
:1011C000A8501C6E030EA96EA69CA69EA680A850D1
:1011D0001B6E040EA96EA69CA69EA680A8501A6E31
:1011E000050EA96EA69CA69EA680A850196E130E89
:1011F000A96EA69CA69EA680A850246E140EA96E69
:10120000A69CA69EA680A850236E150EA96EA69C2D
:10121000A69EA680A850226E160EA96EA69CA69E1B
:10122000A680A850216E170EA96EA69CA69EA68029
:10123000A850286E180EA96EA69CA69EA680A8503F
:10124000276E190EA96EA69CA69EA680A850266E93
:101250001A0EA96EA69CA69EA680A850256E060E04
:10126000A96EA69CA69EA680A8500101186F000139
:1012700012EC02F001011851015CD8A403D0000166
:1012800046EF09F00001000E47EF09F0010E016E74
:10129000000C3A50010170273B50712371515E08D8
:1012A000D8A003D0000161EF09F0000101017051E5
:1012B000016EE70E7125036E0150706F000103C0CF
:1012C00071F1070E0101746F400E756F000188EC1B
:1012D00007F0080E0101746F000170C175F188EC10
:1012E00007F071C172F1090E0101746F000172C142
:1012F00075F188EC07F06C6A000C416A41C040F05F
:101300003F6A40C03EF0149C299A0101716B706BDA
:10131000000149EC09F0000C9EAA9DEF09F0ABB466
:1013200099EF09F0ABB299EF09F0010E016E9FEF52
:1013300009F0AB98AECF20F1AB88000E016EEBEF59
:1013400009F001011651CF5C156F15517908D8A02D
:1013500003D00001B8EF09F00001102AD8B4112A17
:101360007A0E01011627010E016E0001BAEF09F095
:10137000000E016EBFEF09F00400A1EF09F0000CB0
:101380009EBADAEF09F0ABB4C9EF09F0ABA2DAEF1D
:1013900009F0ABB4CFEF09F0ABA2D7EF09F0AB98EF
:1013A000AECF20F1AB88000E016EDCEF09F0040037
:1013B000C0EF09F0AE50016E1BEF0AF001011C6B8B
:1013C000010E216F1D0E206F236B226B000145EC77
:1013D00007F08CEF09F00152D8A419EF0AF00101CF
:1013E0001A511B11D8A403D0000115EF0AF0000117
:1013F000010E0101216F1D0E206F00011BC123F1A1
:101400001AC122F145EC07F00152D8B415EF0AF0E9
:10141000420E01011C25E96EEA6AD8B0EA2AEF6A99
:101420001C51016E0001C3EF0AF0BCEC09F0E9EFBA
:1014300009F0C0EF09F001C01FF101011F511F08A1
:10144000D8A003D000012FEF0AF0000101011F51C5
:101450007F08D8B403D000018BEF0AF0000101012E
:101460001F511B08D8B403D000013FEF0AF0000160
:1014700001011C6B0001B1EF0AF089EF0AF00101D4
:101480001F510D08D8B403D000015DEF0AF0000130
:1014900001011A511B11D8A403D0000159EF0AF021
:1014A000000101011C53D8A403D000015BEF0AF036
:1014B0000001B1EF0AF089EF0AF001011F5108089D
:1014C000D8A403D000016FEF0AF0000101011F5101
:1014D0007F08D8B403D0000189EF0AF000010101B0
:1014E0001C53D8A403D0000189EF0AF000010101C8
:1014F0001C07080E00019EA87BEF0AF0AD6E200EBF
:101500009EA880EF0AF0AD6E080E9EA885EF0AF047
:10151000AD6EAFEF0AF001011C512808D8B003D01E
:101520000001AFEF0AF0000101011C511C2B420F1A
:10153000E96EEA6AD8B0EA2A00011FC1EFFF010193
:101540001A511B11D8B403D00001AFEF0AF000010B
:1015500001011F5100019EA8ABEF0AF0AD6EE9EF4B
:1015600009F0420E01011C25E96EEA6AD8B0EA2AA8
:10157000EF6A3D6A00011CC13CF03CC040F0010133
:101580001C51016E0001C5EF0CF001017053D8B47D
:1015900003D00001CFEF0AF0000108EF0BF0070EB7
:1015A0000101746F400E756F000188EC07F00A0EA0
:1015B0000101746F000170C175F188EC07F00B0E2A
:1015C0000101746F756B000188EC07F00101746B09
:1015D0000A0E756F000188EC07F0100E816EFF0E89
:1015E000956E010170517007000AD8A403D0000164
:1015F00008EF0BF0000184904050402A420FE96E42
:10160000EA6AD8B0EA2A83CFEFFF8480F1EF0AF0CC
:10161000000C415001016A5DD8A003D000013DEFEC
:101620000BF000016AC16CF14050415CD8B039EF59
:101630000BF001016C516C2B420F016E036AD8B0A4
:10164000032A0150716F000103C072F14150412A19
:10165000420FE96EEA6AD8B0EA2AEF500101746FCE
:10166000000172C1EAFF71C1E9FF74C1EFFF14EF1D
:101670000BF06CC140F06AC141F03E503C5C01018E
:101680006E6F3F503D586F6F6F53D8B403D0000159
:101690005BEF0BF0000101016B516E5DD8A003D030
:1016A00000015BEF0BF000016FC103F001016E510F
:1016B00000015EEF0BF001016B51000101016B6F46
:1016C0002A0ED88040546B5DD8A403D0000174EF7B
:1016D0000BF0D8B003D0000174EF0BF000012A0E1C
:1016E000D880405477EF0BF001016B5100010101EC
:1016F0006B6F00016BC16DF101016D53D8A403D074
:10170000000192EF0BF000016C52D8B48EEF0BF099
:101710003FC071F13EC070F149EC09F06BC170F14E
:10172000C5EC0AF001016B51016E0001000C405044
:10173000415CD8A0A4EF0BF00A0E01016A6F2A0EDB
:101740006B6F000109EC0BF04050415CD8A0ADEF8D
:101750000BF0000E016ED0EF0BF04150412A420F0A
:10176000E96EEA6AD8B0EA2AEF500101696F3E2AB1
:10177000D8B43F2A29AA03D00001C4EF0BF000011E
:1017800069C16FF15BEC08F068C103F001016751BA
:10179000E96E000103C0EAFF69C1EFFF010E016EAF
:1017A000000C4152D8B4EBEF0BF03E503F10D8B4D0
:1017B000EBEF0BF04106420E4124E96EEA6AD8B025
:1017C000EA2A20C1EFFF3E50D8B43F063E06010E84
:1017D000016EEDEF0BF0000E016E85EF0CF00101D4
:1017E0001C6B1D6B1F6B0001010E0101686F1E0E4B
:1017F000676F000197EC0BF00152D8B489EF0CF041
:1018000001011E512F08D8A003D000012BEF0CF0CE
:10181000000101011E513908D8B003D000012BEF9F
:101820000CF0000101011F2B300E1E5F1C35206FD4
:101830001D35216F203721372037213720372137B9
:10184000F00E20171E5120251C6F000E21211D6F48
:10185000000187EF0CF001011E514008D8A003D011
:10186000000156EF0CF0000101011E514608D8B0EE
:1018700003D0000156EF0CF0000101011F2B370EC1
:101880001E5F1C35206F1D35216F20372137203713
:10189000213720372137F00E20171E5120251C6FCD
:1018A000000E21211D6F000187EF0CF001011E5178
:1018B0006008D8A003D0000181EF0CF00001010105
:1018C0001E516608D8B003D0000181EF0CF0000172
:1018D00001011F2B570E1E5F1C35206F1D35216F18
:1018E000203721372037213720372137F00E2017B6
:1018F0001E5120251C6F000E21211D6F000187EF56
:101900000CF01EC120F1D1EF0BF089EF0CF0F4EFD9
:101910000BF01BC103F001011A51E96E000103C075
:10192000EAFF1DC1ECFFED521CC1EFFF01011F5387
:10193000D8B403D00001A1EF0CF00001000EA2EF1B
:101940000CF0010E016ED1EF0CF001011A6B0001D9
:1019500001011A5100013FEC00F001011A2B0001B6
:101960009EA8B0EF0CF0AD6E0E0E01011A5DD8B45A
:1019700003D00001A8EF0CF000017DEC09F001019B
:101980001B6B1A6B0001DEEF09F00152D8B4D9EFDE
:101990000CF0010E01011B6F180E1A6F0001EFEF22
:1019A0000BF00152D8B4D9EF0CF019C136F018C1C0
:1019B00037F00D0E9EA8DAEF0CF0AD6E0A0E9EA861
:1019C000DFEF0CF0AD6E01011B6B190E1A6FC00E2C
:1019D0001C6FA80E1D6F1E6B020E1F6F0001EBEC3B
:1019E00001F001011B6B210E1A6FFF0E1C6FFF0E21
:1019F0001D6FFF0E1E6F1F6B0001EBEC01F001016C
:101A00001B6B250E1A6FC00E1C6FA80E1D6F1E6B70
:101A1000010E1F6F0001EBEC01F033EC02F0010E40
:101A2000016E87EF3EF0D89001015535566FB40E28
:101A3000576F000E926E8996010E586F00010101DA
:101A400058512008D8B003D0000130EF0DF000014C
:101A50008982899489840101582B00011FEF0DF0C0
:101A6000010E0101586F0001010158512F08D8B033
:101A700003D0000180EF0DF00001010158510F0863
:101A8000D8B003D0000154EF0DF00001D89001014F
:101A900056375737D8A003D0000153EF0DF000019F
:101AA000899254EF0DF089828994010158510F08F1
:101AB000D8A003D000016BEF0DF0000180B264EFFD
:101AC0000DF0D89065EF0DF0D88001015B375C37E1
:101AD0005D375E3700018984010158510F08D8B481
:101AE00003D000017BEF0DF00001020E926E89948D
:101AF0008984899489840101582B000134EF0DF009
:101B00005BC100F05CC101F05DC102F05EC103F099
:101B1000000C0101586B596B57355A6F5A37FC0E40
:101B20005A17060E5B6F010E5C6F000101015C51DC
:101B30000508D8B003D00001ABEF0DF00001D8903C
:101B40000101583759375A375B37000101015C2BC7
:101B5000000196EF0DF08986010E01015C6F000116
:101B600001015C511908D8B003D00001E4EF0DF079
:101B70000001D8900101583759375A375B37D8A040
:101B800003D00001C8EF0DF000018992C9EF0DF0FC
:101B900089828984899401015C510908D8A003D005
:101BA0000001DFEF0DF0000180B0DAEF0DF0D8900A
:101BB000DBEF0DF0D88001015F37603700010101D4
:101BC0005C2B0001B0EF0DF0899601015F51016EB1
:101BD0006051026E0001000C080E016E000004004E
:101BE0008B9694960400010164378298D8B094884B
:101BF000D8A094989486000182A6FCEF0DF0012EE7
:101C0000EEEF0DF004008B9694960000948804008B
:101C10000400948682A60AEF0EF0016A040082B8DE
:101C200001808B96949682989498000C080E01017E
:101C3000686F000100C069F194880400948682A650
:101C40001FEF0EF082B8D88082A8D8900136040029
:101C500094968B960101682F02D004D000010001F8
:101C60001CEF0EF09488040082986951D8A49498CF
:101C700000010000948682A63BEF0EF004008B96D4
:101C80009496040082989498000C010E0101556FFF
:101C90000001E76B9488040094860400829894986D
:101CA00004008B969496A00E0101646F0001ECEC89
:101CB0000DF00101646B0001ECEC0DF00101646BAF
:101CC0000001ECEC0DF094980000948682A666EF7B
:101CD0000EF00400000000000000948804009488C6
:101CE0000400948604008298949804008B9694963D
:101CF000A10E0101646F0001ECEC0DF00101566BC7
:101D00000001010156510608D8B003D000019DEF33
:101D10000EF00001D40E01015625E96EEA6AD8B032
:101D2000EA2A010E006E000116EC0EF00150EF6E73
:101D30000101562B000181EF0EF0D43DAAEF0EF009
:101D4000D53DAAEF0EF0006A16EC0EF015EF0FF07D
:101D5000FBEF0EF00101556B566B0001010156516E
:101D60000B08D8B003D00001F4EF0EF00001580EBC
:101D700001015625E96E010EEA6ED8B0EA2A5651E5
:101D80000A08D8A003D00001CAEF0EF00001000E2F
:101D9000CBEF0EF0010E0101666F000166C100F08D
:101DA00016EC0EF001C057F157C1EFFF070E01010D
:101DB0005625016E036AD8B0032A0150D40FE96E8C
:101DC000000E0320EA6EEF50575DD8A403D0000147
:101DD000EFEF0EF00001010E0101556F000101014E
:101DE000562B0001AEEF0EF0DB53D8A4FBEF0EF044
:101DF0000101556B000194980000948682A6FEEFC5
:101E00000EF0040000000000000094880400E72B9E
:101E1000E7516308D8A015EF0FF001015553D8B46E
:101E200003D000016FEF0EF0000101015553D8A45B
:101E300003D000011FEF0FF00001D56BD46B01013F
:101E40005553D8A403D000012AEF0FF00001000E73
:101E50002BEF0FF0010E016E000C0101186B000159
:101E60000101185100017FEC01F00101182B000164
:101E70009EA838EF0FF0AD6E060E0101185DD8B4C4
:101E800003D0000130EF0FF0030E196F0001390E7F
:101E90009EA848EF0FF0AD6E0101192F02D004D0BB
:101EA0000001000147EF0FF0060E1A6F000101015B
:101EB0001A5100017FEC01F001011A2B00019EA8CC
:101EC0005FEF0FF0AD6E0C0E01011A5DD8B403D0B8
:101ED000000157EF0FF0070E1B6F00012E0E9EA89A
:101EE0006FEF0FF0AD6E01011B2F02D004D0000187
:101EF00000016EEF0FF0556B000113EC0DF003C005
:101F00001BF102C01AF101C019F100C018F1010162
:101F100018512008D8B403D00001AAEF0FF0000137
:101F2000010119511108D8B403D00001AAEF0FF034
:101F3000000101011A510208D8B403D00001AAEF30
:101F40000FF0000101011B53D8A403D00001DAEF08
:101F50000FF000010101556B000113EC0DF003C0FF
:101F60001FF102C01EF101C01DF100C01CF10101F2
:101F70001C512108D8B403D00001F4EF0FF0000188
:101F800001011D511108D8B403D00001F4EF0FF086
:101F9000000101011E510208D8B403D00001F4EF82
:101FA0000FF0000101011F53D8B403D00001F4EF7A
:101FB0000FF000010101186B00010101185100012F
:101FC0008EEC01F00101182B00019EA8E5EF0FF047
:101FD000AD6E050E0101185DD8B403D00001DDEF30
:101FE0000FF000010CEF10F00101186B000101016E
:101FF0001851000199EC01F00101182B00019EA875
:10200000FFEF0FF0AD6E090E0101185DD8B403D0DB
:102010000001F7EF0FF000010101186B0001010151
:1020200018510001A6EC01F00101182B00019EA837
:1020300017EF10F0AD6E0D0E0101185DD8B403D08E
:1020400000010FEF10F0090E196F00012E0E9EA86F
:1020500027EF10F0AD6E0101192F02D004D000015E
:10206000000126EF10F0010E926E000190EC03F0DB
:102070000101576B000189EC0DF002C019F101C09C
:1020800018F1010118515408D8B403D000016DEFC4
:1020900010F00001010119514108D8B403D000012A
:1020A0006DEF10F000010101186B000101011851E2
:1020B00000018EEC01F00101182B00019EA85EEFDB
:1020C00010F0AD6E050E0101185DD8B403D000010B
:1020D00056EF10F0000185EF10F00101186B0001C0
:1020E00001011851000199EC01F00101182B0001C8
:1020F0009EA878EF10F0AD6E090E0101185DD8B4FE
:1021000003D0000170EF10F000010101186B000115
:10211000010118510001B5EC01F00101182B00017B
:102120009EA890EF10F0AD6E0F0E0101185DD8B4AF
:1021300003D0000188EF10F0070E196F00012E0E7A
:102140009EA8A0EF10F0AD6E0101192F02D004D0AF
:10215000000100019FEF10F0070E716F0001B5EC58
:1021600007F00150800B000AD8A4D1EF10F0010154
:10217000186B000101011851000199EC01F00101F7
:10218000182B00019EA8C2EF10F0AD6E090E0101E0
:10219000185DD8B403D00001BAEF10F00001E9EFE8
:1021A00010F00101186B00010101185100018EECC3
:1021B00001F00101182B00019EA8DCEF10F0AD6EBC
:1021C000050E0101185DD8B403D00001D4EF10F062
:1021D00000010101186B0001010118510001C5EC5B
:1021E00001F00101182B00019EA8F4EF10F0AD6E74
:1021F0000F0E0101185DD8B403D00001ECEF10F010
:10220000070E196F00012E0E9EA804EF11F0AD6E9F
:102210000101192F02D004D00001000103EF11F0D9
:10222000000145EC0EF0E753D8A431EF11F00101A5
:10223000186B000101011851000199EC01F0010136
:10224000182B00019EA822EF11F0AD6E090E0101BE
:10225000185DD8B403D000011AEF11F0000149EF66
:1022600011F00101186B00010101185100018EEC01
:1022700001F00101182B00019EA83CEF11F0AD6E9A
:10228000050E0101185DD8B403D0000134EF11F040
:102290000001D2EF3EF0FF0E956E816AF19E200E96
:1022A000936E8480848284849690969296945BEF59
:1022B00011F04BEF11F0020E0101646F0001D5EC3B
:1022C00001F08494020E0101646F0001D5EC01F06D
:1022D0001F0E0101716F0001B5EC07F001C01CF188
:1022E0001F0E0101746F00011CC175F188EC07F02D
:1022F000020E0101646F0001D5EC01F0070E01012F
:10230000716F0001B5EC07F00150800B000AD8A4F2
:10231000A6EF11F001011C6B000101011C5100012D
:1023200002EC00F001011C2B00019EA895EF11F0BA
:10233000AD6E0E0E01011C5DD8B403D000018DEF0F
:1023400011F0000E016E000188EF12F00101746BB4
:10235000210E756F000188EC07F0020E0101646F19
:102360000001D5EC01F00E0E0101746F480E756F7F
:10237000000188EC07F00A0E0101746F756B000113
:1023800088EC07F00B0E0101746F756B000188EC8F
:1023900007F00C0E0101746F200E756F000188ECC0
:1023A00007F00D0E0101746F020E756F000188ECCD
:1023B00007F0040E0101746F400E756F000188EC88
:1023C00007F0010E0101746F460E756F000188EC75
:1023D00007F0020E0101746F5F0E756F000188EC4B
:1023E00007F0030E0101746F5E0E756F000188EC3B
:1023F00007F0070E0101746FFF0E756F000188EC86
:1024000007F00F0E0101746F756B000188EC07F087
:102410000101746B610E756F000188EC07F0020E0C
:102420000101646F0001D5EC01F001011B6B00019B
:1024300001011B510508D8B003D0000139EF12F09B
:102440000001010E01011B251C6F320E1B25E96ED8
:10245000EA6AD8B0EA2A0001EFCF1DF11CC174F17D
:102460001DC175F188EC07F001011B2B000118EF6D
:1024700012F001011B6B000101011B510708D8B0CC
:1024800003D0000157EF12F00001080E01011B25D7
:102490001C6F00011CC174F1FF0E0101756F00017A
:1024A00088EC07F001011B2B00013CEF12F0070E36
:1024B0000101746F470E756F000188EC07F0470E3D
:1024C000386E0101746B200E756F000188EC07F007
:1024D0000C0E0101746F040E756F000188EC07F09B
:1024E0000D0E0101746F756B000188EC07F0070E8B
:1024F0000101746FFF0E756F000188EC07F0010198
:10250000746B220E756F000188EC07F0010E016EEE
:10251000000C016A026A006A036A01017251D8B4B0
:1025200003D000019BEF12F07151D8A403D0000139
:10253000C6EF12F00001100E0101736F0001D89078
:1025400001016F377037003603367251035CD8B41F
:1025500003D00001AFEF12F07151005C0001D8A070
:10256000BBEF12F001017151005ED8A00306725159
:10257000035ED8800001013602360101732F02D0BC
:1025800004D0000100019FEF12F000010000000CD8
:102590000101666B000101016651662B670FE96E50
:1025A000010EEA6ED8B0EA2A000164C170F163C17D
:1025B0006FF10101726B0A0E716F000189EC12F06C
:1025C0000050300FEF6E64C170F163C16FF1010113
:1025D000726B0A0E716F000189EC12F002C064F197
:1025E00001C063F1010163516411D8B403D000014B
:1025F000CBEF12F0000166C165F101016653D8A46A
:1026000003D0000117EF13F0000101016607670E08
:102610006625E96E010EEA6ED8B0EA2A0001EFCF16
:102620006CF16CC16DF1AEEC08F0FDEF12F0010140
:102630006551016E0001000C298629842998010149
:102640001D6B000101011D51000143EC01F001016E
:102650001D2B00019EA82AEF13F0AD6E0D0E010197
:102660001D5DD8B403D0000122EF13F0646B0001AC
:102670001CC063F1C8EC12F02E0E01016D6F000159
:10268000AEEC08F00101646B00011BC063F1C8EC03
:1026900012F02E0E01016D6F0001AEEC08F0010189
:1026A000646B00011AC063F1C8EC12F02E0E010138
:1026B0006D6F0001AEEC08F00101646B000119C000
:1026C00063F1C8EC12F0000C2986298429980101D5
:1026D0001D6B000101011D51000152EC01F00101CF
:1026E0001D2B00019EA872EF13F0AD6E0B0E0101C1
:1026F0001D5DD8B403D000016AEF13F0646B0001D4
:1027000024C063F1C8EC12F02E0E01016D6F0001C0
:10271000AEEC08F00101646B000123C063F1C8EC6A
:1027200012F02E0E01016D6F0001AEEC08F00101F8
:10273000646B000122C063F1C8EC12F02E0E01019F
:102740006D6F0001AEEC08F00101646B000121C067
:1027500063F1C8EC12F0000C298629842998010144
:102760001D6B000101011D51000160EC01F0010130
:102770001D2B00019EA8BAEF13F0AD6E0E0E0101E5
:102780001D5DD8B403D00001B2EF13F0646B0001FB
:1027900028C063F1C8EC12F02E0E01016D6F00012C
:1027A000AEEC08F00101646B000127C063F1C8ECD6
:1027B00012F02E0E01016D6F0001AEEC08F0010168
:1027C000646B000126C063F1C8EC12F02E0E01010B
:1027D0006D6F0001AEEC08F00101646B000125C0D3
:1027E00063F1C8EC12F0000C010120AF03D000012E
:1027F00013EF14F00F0E006E1F3900160A0E005C66
:10280000D8A003D000010AEF14F0300E002600011A
:102810000EEF14F0010120510026000100509EA887
:102820000FEF14F0AD6E0F0E01011F170A0E1F5DA2
:10283000D8A003D0000121EF14F0300E000125EFE5
:1028400014F00101209F2051000101011F271F5199
:1028500000019EA829EF14F0AD6E000C01011E6B63
:10286000000101011E51000170EC01F001011E2B5D
:1028700000019EA839EF14F0AD6E0C0E01011E5D33
:10288000D8B403D0000131EF14F01D6B0001010139
:102890001D510408D8B003D000016CEF14F0000102
:1028A000320E01011D25E96EEA6AD8B0EA2A00015C
:1028B000EFCF1EF11EC11FF1370E0101206F000185
:1028C000F4EC13F03A0E9EA863EF14F0AD6E010124
:1028D0001D2B000147EF14F037C01FF1370E010127
:1028E000206F0001F4EC13F0200E9EA875EF14F099
:1028F000AD6E000C21C124F10101256B000120C146
:1029000003F0000E01012411226F03502511236FE3
:102910002251016E2351026E0001000C01011F6B58
:102920001D51000B006E1E51800B036E00500310F2
:10293000D8A403D00001ADEF14F0000101011F5332
:10294000D8A403D00001A9EF14F00001000EAAEFF3
:1029500014F0010E01011F6F000101011D51000B58
:10296000006E1E51400B036E00500310D8A403D01C
:102970000001CBEF14F0000101011F53D8A403D0D4
:102980000001C7EF14F00001000EC8EF14F0010EB3
:1029900001011F6F000101011D51000B006E1E514E
:1029A000100B036E00500310D8A403D00001E9EF10
:1029B00014F0000101011F53D8A403D00001E5EF7A
:1029C00014F00001000EE6EF14F0010E01011F6F7C
:1029D000000101011D51080B006E1E51000B036E1A
:1029E00000500310D8A403D0000107EF15F0000138
:1029F00001011F53D8A403D0000103EF15F000011B
:102A0000000E04EF15F0010E01011F6F000101011E
:102A10001D511D25206F1E511E21216F1F51202584
:102A2000016E000E2121036E0350026E00012BEF98
:102A300015F001011C6B000101011C510708D8B001
:102A400003D0000134EF15F000011BC11EF11AC1C3
:102A50001DF18EEF14F002C01BF101C01AF101014B
:102A60001C2B00011CEF15F001011A51016E1B51C6
:102A7000026E00014DEF19F0010121510408D8A0A8
:102A800003D0000156EF15F00001FF0AD8A452EF61
:102A900015F001012051DC08D8A003D0000156EF49
:102AA00015F00001000E016E64EF15F030EC08F037
:102AB00021C170F020C16FF070C072F16FC071F170
:102AC00094EC07F0010E016E000C030E01012025AD
:102AD000E96E000E2121EA6E0001EFCF22F122C142
:102AE0006EF182EC08F0020E01012025E96E000E65
:102AF0002121EA6E0001EFCF22F122C16EF182ECBA
:102B000008F0010E01012025E96E000E2121EA6E78
:102B10000001EFCF22F122C16EF182EC08F0010139
:102B20002051E96E2151EA6E0001EFCF22F122C15E
:102B30006EF182EC08F0000C01011E511E07000A24
:102B4000D8A403D00001ADEF15F0000101016E6BB8
:102B5000000182EC08F09CEF15F0000C01012551FA
:102B6000036E2451D8B4250724070310D8A403D03A
:102B70000001CFEF15F0000101012351036E225136
:102B8000222BD8B4232BE96E000103C0EAFFEFCF5C
:102B900026F126C16EF182EC08F0AEEF15F0000CC4
:102BA00021C122F122C16EF182EC08F020C16EF148
:102BB00082EC08F0000C030E01012025E96E000EE6
:102BC0002121EA6E0001EFCF22F122C16FF15BEC0F
:102BD00008F0020E01012025E96E000E2121EA6EA7
:102BE0000001EFCF22F122C16FF15BEC08F0010E82
:102BF00001012025E96E000E2121EA6E0001EFCFD0
:102C000022F122C16FF15BEC08F001012051E96E65
:102C10002151EA6E0001EFCF22F122C16FF15BEC8E
:102C200008F0000C2B6A2BC02AF02990450E0101F8
:102C30006E6F000182EC08F001016E6B000182EC06
:102C400008F0C2C021F1C1C020F1D0EC15F00101A3
:102C50006E6B000182EC08F0C52BC5C06EF182ECF2
:102C600008F00101216B206B0001D0EC15F0640E1F
:102C700001016E6F000182EC08F0AEC06EF182ECD3
:102C800008F00101216B190E206F0001DBEC15F03B
:102C90000101216BB30E206F0001DBEC15F02A500F
:102CA0000101206F201F000120C16EF182EC08F0AD
:102CB0002B500101206F201F000120C16EF182EC1A
:102CC00008F00101216B190E206F000165EC15F071
:102CD0000101216BB30E206F000165EC15F0000CB3
:102CE00022C123F10101246B000123C16FF15BECD0
:102CF00008F021C16FF15BEC08F0000C2990C3C013
:102D00002AF0C4C02BF0B8C021F1B7C020F1D0EC3C
:102D100015F0BAC021F1B9C020F1D0EC15F0E9C02E
:102D200021F1E8C020F1D0EC15F00101216B190E62
:102D3000206F0001DBEC15F00101216BB30E206F59
:102D40000001DBEC15F001016F6B00015BEC08F09A
:102D5000110E01016F6F00015BEC08F0E9C022F178
:102D6000E8C021F170EC16F029AEBBEF16F0FF0EB3
:102D70002B6E2BC02AF02A500101206F201F00016A
:102D800020C16EF182EC08F02B500101206F201F52
:102D9000000120C16EF182EC08F070EF17F06EC0F8
:102DA00021F16DC020F130EC08F0FF0E0101726FCF
:102DB000F20E716F000194EC07F0716A0101236B50
:102DC000A60E226F256B060E246F0001AEEC15F0E7
:102DD0000101236B320E226F256B060E246F00015A
:102DE000AEEC15F0ADC022F122C16EF182EC08F01C
:102DF000ACC06EF182EC08F00E0E01012027000E2F
:102E000021230001C2EC07F001012153D8B403D003
:102E100000011AEF17F00001010120513B08D8B062
:102E200003D000011AEF17F000010101216B3C0EE5
:102E3000206F0001050E0101746F000120C175F1C2
:102E400088EC07F021C122F1060E0101746F000128
:102E500022C175F188EC07F00101746B240E756FC7
:102E6000000188EC07F0000C30EC08F02AC0C3F039
:102E70002BC0C4F001011F6B1E6B7052D8B403D07D
:102E8000000149EF17F000016F501C08D8B051EF56
:102E900017F01C0E6F5C01011E6F000E70581F6F43
:102EA0000001080E01011E250001E86F000E01015E
:102EB0001F210001E96F140EE825C16F000EE92102
:102EC000C26F0101216B206B00013CEC15F0080E74
:102ED000AD6FAC6B110EAE6F12EC16F07EEF16F00C
:102EE000CFEC16F0000C299629942988080EAD6FB6
:102EF000AC6B110EAE6FB86B440EB76FBA6B430E6E
:102F0000B96F0101216B1C0E206F00013CEC15F024
:102F1000010E01016E6F000182EC08F0010E01014B
:102F20006E6F000182EC08F0060E01016E6F000169
:102F300082EC08F001016E6B000182EC08F00101E7
:102F4000216BFF0E206F000165EC15F0040E0101EE
:102F50001E6F00019CEC15F00101216B190E206F12
:102F6000000165EC15F00C0E01011E6F00019CECD8
:102F700015F00101236B320E226F256B060E246FB4
:102F80000001AEEC15F070500108D8A0D7EF17F093
:102F9000D8A4D0EF17F06F500708D8A0D7EF17F0DC
:102FA00001016E6B000182EC08F0C3EF17F0630EB5
:102FB00001016E6F000182EC08F0820E01016E6F5C
:102FC000000182EC08F0530E01016E6F000182ECEB
:102FD00008F0630E01016E6F000182EC08F0350EFF
:102FE00001016E6F000182EC08F0010E01016E6FAD
:102FF000000182EC08F001011A510F0B1E6F000155
:103000001EC16EF182EC08F03D0E01016E6F0001F1
:1030100082EC08F0070E01016E6F000182EC08F0EF
:10302000010E01016E6F000182EC08F00101236BBB
:10303000320E226F256B060E246F0001AEEC15F0E8
:103040000C0E01016E6F000182EC08F02998036AF2
:10305000360EE96E03C0EAFFECCF1FF1ED52EFCF61
:103060001EF11FC121F11EC120F17AEC14F002C043
:103070001DF101C01CF11DC164F11CC163F1C8EC5C
:1030800012F001C01BF12988060E01011B251E6FDD
:1030900000011EC16EF182EC08F0000E81BA010E33
:1030A000000AD8A46AEF18F001011E6B00010101AB
:1030B0001E51000104EC01F00009D8B468EF18F0CB
:1030C00001011E2B6E6F000182EC08F057EF18F023
:1030D0007EEF18F001011E6B000101011E5100017D
:1030E00010EC01F00009D8B47EEF18F001011E2B9E
:1030F0006E6F000182EC08F06DEF18F01DC164F1F5
:103100001CC163F1C8EC12F001011A510308D8B4D4
:1031100003D00001B4EF18F00001360E01016E6F0C
:10312000000182EC08F0040E01016E6F000182ECD8
:1031300008F0010E0101216F090E206F000165ECFE
:1031400015F0320E01016E6F000182EC08F0040EE2
:1031500001016E6F000182EC08F00101216BFB0E92
:10316000206F000165EC15F0370E01016E6F000154
:1031700082EC08F0040E01016E6F000182EC08F091
:10318000010E01016E6F000182EC08F00F0E0101CB
:103190006E6F000182EC08F0030E01016E6F0001FA
:1031A00082EC08F0060E01016E6F000182EC08F05F
:1031B000FF0E01016E6F000182EC08F001011A514F
:1031C0001308D8B403D00001FFEF18F00001EA6A39
:1031D000A60EE96E010EE26E030EE16E060E016EA2
:1031E000E6CFEEFF012EF0EF18F00CC1B6F00BC1E8
:1031F000B5F00AC1B4F009C1B3F013EF19F0060E2F
:10320000016EEA6AA60EE96EFF0EEE6E012E04EF65
:1032100019F0040E016EEA6AB30EE96EFF0EEE6E4F
:10322000012E0EEF19F034EC17F0C6EF19F0EC5345
:10323000D8A46FEF19F01C6A1B6A1A6A196A036A2C
:10324000360EE96E03C0EAFFECCF1BF1ED52EFCF73
:103250001AF11BC121F11AC120F17AEC14F002C05D
:1032600019F101C018F1F66BF56B0101216BED0E40
:10327000206F236B226B000145EC07F00101216BED
:10328000EF0E206F236B226B000145EC07F019C194
:103290001BF118C11AF119EF15F002C01BF101C0A2
:1032A0001AF101011A511F0B006E1B51000B036E26
:1032B0000050140F0001F16F000E0320F26FF2C0F6
:1032C000F4F0F1C0F3F019C100F118C1FFF0F4C03F
:1032D00002F1F3C001F1010EEC6FD7EF19F0EC2D04
:1032E00074EF19F07EEF19F0EC510308D8B47EEFBB
:1032F00019F0EC511308D8A4D7EF19F00101216B94
:10330000ED0E206F0001F2C023F1F1C022F145EC77
:1033100007F00152D8B4D7EF19F001011A6B000180
:1033200001011A510001F2EC00F001011A2B000119
:103330009EA898EF19F0AD6E120E01011A5DD8B477
:1033400003D0000190EF19F0060E1B6F00012E0E46
:103350009EA8A8EF19F0AD6E01011B2F02D004D07A
:1033600000010001A7EF19F0010E16262B6A0001DB
:103370002BC02AF02A52D8A4C1EF19F02990C2EF2D
:1033800019F02980ECC01AF173EF17F0F25104081C
:10339000D8A0D7EF19F0D8A4D3EF19F0F151AF08A6
:1033A000D8A0D7EF19F0F351F127F451F223EC51E3
:1033B0003008D8B4E1EF19F0EC511308D8A416EF97
:1033C0001AF00101216BEF0E206F236B140E226F98
:1033D000000145EC07F00152D8B412EF1AF0F52BBA
:1033E000D8B4F62BF951F55DD8A404EF1AF0FA51D0
:1033F000F65DD8A404EF1AF0F4C0F2F0F3C0F1F0D7
:10340000130EEC6F12EF1AF0F851F65DD8A012EF20
:103410001AF0D8A411EF1AF0F751F55DD8A012EF09
:103420001AF0EC6B010E016E18EF1AF0000E016E2F
:1034300075EF3FF00101206B216B0001010121516B
:103440001E5DD8B003D000015CEF1AF00001D8A4D3
:1034500033EF1AF001011D51205DD8A003D0000107
:103460005CEF1AF00001010E0101686F1F0E676F1B
:10347000000197EC0BF00152D8B45CEF1AF0010197
:103480001B511C11D8A403D0000155EF1AF0000104
:1034900001011C51036E1B511B2BD8B41C2BE96E70
:1034A000000103C0EAFF1FC1EFFF0101202BD8B4C8
:1034B000212B00011EEF1AF001012051016E215154
:1034C000026E0001000C01011C515E08D8A003D05F
:1034D000000173EF1AF00001E70E01011C251C6FBB
:1034E000000180EF1AF001011C514508D8B003D04B
:1034F000000180EF1AF00001190E01011C270001E4
:1035000001011C51016E0001000C3D6A3C6A070E6E
:103510000101716F0001B5EC07F00150100B000ABA
:10352000D8B49AEF1AF02E0E9EA894EF1AF0AD6E52
:1035300059EC11F00101746B600E756F000188EC9D
:1035400007F0070E0101716F0001B5EC07F00101F2
:10355000196B000101C018F10101746B200E756F29
:10356000000188EC07F038500101185DD8B403D091
:103570000001C4EF1AF0000101011953D8A403D0CF
:10358000000174EF1BF0000138C039F001011C6B21
:10359000000138C01BF11BC13BF03A6A7DEC09F019
:1035A000120E0101706F0001C5EC0AF001011C6BE5
:1035B0009C0E1B6F1E6B120E1D6F00011AEC1AF091
:1035C000120E3A26000E3B227DEC09F09FC03DF022
:1035D0009EC03CF09C51010B000AD8B416EF1BF0C2
:1035E0003D52D8A4F9EF1AF03C503F08D8B016EF7E
:1035F0001BF03D500508D8A016EF1BF0D8A406EF2D
:103600001BF03C50EE08D8A016EF1BF0120E3C5EEB
:10361000000E3D5AADC021F1ACC020F17AEC14F09F
:1036200002C0ADF001C0ACF030EF1BF03D6A3C6A67
:1036300001011B6B000101011B51000112EC00F0A4
:1036400001011B2B00019EA823EF1BF0AD6E0D0E98
:1036500001011B5DD8B403D000011BEF1BF000017A
:103660009D514508D8B03EEF1BF09D515E08D8A093
:103670003EEF1BF09DC038F061EF1BF03D6A3C6AE5
:1036800001011B6B000101011B51000121EC00F045
:1036900001011B2B00019EA84BEF1BF0AD6E0D0E20
:1036A00001011B5DD8B403D0000143EF1BF0010EF4
:1036B00038241B6F00011BC11CF163EC1AF001C020
:1036C00038F0010E385C01011B6F00011BC11CF1B9
:1036D00063EC1AF001C01AF1030E0101746F0001CE
:1036E0001AC175F188EC07F03C52D8A47FEF1BF0AB
:1036F0003D52D8A47FEF1BF0000E80EF1BF0010EAF
:10370000016E8DEF3FF0716A6E6A71C06DF06EC030
:1037100070F06DC06FF02B6A2BC02AF02A52D8A42B
:1037200095EF1BF0299096EF1BF029800101726B39
:10373000716B000194EC07F0000C010E0101686F41
:10374000560E676F000197EC0BF00152D8B4B6EF3C
:103750001BF001015651555DD8B403D00001B6EFFE
:103760001BF00001010E016EB8EF1BF0000E016EA0
:10377000000C010E0101686F200E676F000197ECCD
:103780000BF00152D8B4F3EF1BF0010E0101686F8A
:10379000210E676F000197EC0BF00152D8B4F3EFE4
:1037A0001BF00101256B000120C124F124C127F188
:1037B0000101266B036A21512611226F0350271144
:1037C000236F00011FC103F001011E51E96E0001CA
:1037D00003C0EAFF23C1ECFFED5222C1EFFF010E4F
:1037E000016EF5EF1BF0000E016E000C040E0101DE
:1037F0001F6F030E1D25216F000E1E21226F000179
:1038000022C168F121C167F197EC0BF00152D8B4E5
:1038100042EF1CF0020E01011D25226F000E1E2139
:10382000236F000123C168F122C167F197EC0BF00F
:103830000152D8B442EF1CF0010E01011D25236F87
:10384000000E1E21246F000124C168F123C167F11D
:1038500097EC0BF00152D8B442EF1CF001011D515E
:10386000246F1E51256F000125C168F124C167F145
:1038700097EC0BF00152D8B442EF1CF0010E016E30
:1038800044EF1CF0000E016E000C01011E511F11CF
:10389000D8A403D0000162EF1CF00001010E010169
:1038A000686F200E676F000197EC0BF00152D8B4DF
:1038B00062EF1CF001011E51D8B41F071E07000162
:1038C00045EF1CF001011E53D8B403D0000176EF80
:1038D0001CF0000101011F53D8B403D0000176EFA2
:1038E0001CF00001010E016E78EF1CF0000E016E5D
:1038F000000C030E01011A25E96E000E1B21EA6E71
:103900000001EFCF1CF11CC155F19DEC1BF00152E1
:10391000D8B4C3EF1CF0020E01011A25E96E000EA7
:103920001B21EA6E0001EFCF1DF11DC155F19DEC89
:103930001BF00152D8B4C3EF1CF0010E01011A258F
:10394000E96E000E1B21EA6E0001EFCF1EF11EC1D1
:1039500055F19DEC1BF00152D8B4C3EF1CF00101EE
:103960001A51E96E1B51EA6E0001EFCF1FF11FC122
:1039700055F19DEC1BF00152D8B4C3EF1CF0010EC1
:10398000016EC5EF1CF0000E016EA0EF1DF00101ED
:103990001D6B000183EC1BF001011A2D02D004D035
:1039A00000010001DFEF1CF00001060E016EEA6A63
:1039B000A60EE96EFF0EEE6E012EDAEF1CF001018D
:1039C000216B010E206F0001D0EC15F0080E0101F3
:1039D000216F206B0001D0EC15F0060E01016E6F17
:1039E000000182EC08F0040E01016E6F000182EC10
:1039F00008F001011C6B00011AC11BF11CC121F16F
:103A00001BC120F1D0EC15F00101236B320E226FA7
:103A1000256B060E246F0001AEEC15F00101216B41
:103A2000190E206F000165EC15F00101236BA60E45
:103A3000226F256B060E246F0001AEEC15F001011C
:103A4000216BB30E206F000165EC15F0080EAD6F11
:103A5000060EAC6FCFEC16F0BBEF1DF00101556BFD
:103A600000019DEC1BF00152D8B4F4EF1DF0010EE3
:103A70000101556F00019DEC1BF00152D8B4F4EF29
:103A80001DF0080E0101556F00019DEC1BF0015265
:103A9000D8B4F4EF1DF00101556B00019DEC1BF053
:103AA0000152D8B4F4EF1DF0060E0101556F00016C
:103AB0009DEC1BF00152D8B4F4EF1DF0040E01018F
:103AC000556F00019DEC1BF00152D8B4F4EF1DF0CE
:103AD000010E01011F6F180E1E6F0001B9EC1BF0E3
:103AE0000152D8B4F4EF1DF001011C6BBB0E1B6F2B
:103AF0001E6B060E1D6F00011AEC1AF00150021029
:103B0000D8B4F4EF1DF001011E6BB30E1D6F000160
:103B1000F6EC1BF00152D8B4F4EF1DF001011F6B5D
:103B2000060E1E6F000145EC1CF00152D8B4F4EFF4
:103B30001DF001011B6B190E1A6F000179EF1CF0CB
:103B40000152D8B4F4EF1DF00101182D02D004D0B9
:103B500000010001C1EF1DF0000101011953D8B4AB
:103B600003D00001C1EF1DF00001020E01011A6F28
:103B70000001C7EF1CF0010E016EF6EF1DF0F4EF2F
:103B80001DF0010118510208D8B403D00001F4EF70
:103B90001DF0000101011953D8B403D00001F4EF66
:103BA0001DF000012550B35DD8A4F3EF1DF02650A1
:103BB000B45DD8A4F3EF1DF02750B55DD8A4F3EFA2
:103BC0001DF02850B65DD8A4F3EF1DF0EA6A2C0E64
:103BD000E96EE26ABB0EE16E060E016EE6CFEEFF05
:103BE000012EEEEF1DF0148C000E016EA2EF3FF0DF
:103BF000010E0101686F1D0E676F000197EC0BF05D
:103C00000152D8B408EF1EF0010E016E0AEF1EF04B
:103C1000000E016E000C01011A513E241C6F1B5155
:103C20003F201D6F3D5CD8B003D0000129EF1EF08E
:103C30000001D8A425EF1EF03C5001011C5DD8A066
:103C400003D0000129EF1EF000011DC13DF01CC191
:103C50003CF0415001011A251C6F000E1B211D6F05
:103C60001D53D8B403D0000142EF1EF000014050B4
:103C700001011C5DD8A003D0000142EF1EF000013D
:103C80001CC140F0EBEF1EF02990299A2B6A2BC043
:103C90002AF0450E0101556F00019DEC1BF0015209
:103CA000D8B4EFEF1EF0F8EC1DF00152D8B4EFEFEE
:103CB0001EF001011F6BC10E1E6F0001B9EC1BF05D
:103CC0000152D8B4EFEF1EF001011F6B020E1E6F00
:103CD000000145EC1CF00152D8B4EFEF1EF00101D9
:103CE0001F6B020E1E6F000145EC1CF00152D8B490
:103CF000EFEF1EF0F8EC1DF00152D8B4EFEF1EF01C
:103D00000101686BAE0E676F000197EC0BF001527A
:103D1000D8B4EFEF1EF001011F6B020E1E6F000101
:103D200045EC1CF00152D8B4EFEF1EF001011E6B00
:103D3000B30E1D6F0001F6EC1BF00152D8B4EFEF8B
:103D40001EF001011E6BAF0E1D6F0001F6EC1BF0A3
:103D50000152D8B4EFEF1EF01950AF5DD8A4C0EFF8
:103D60001EF01A50B05DD8A4C0EF1EF01B50B15D1C
:103D7000D8A4C0EF1EF01C50B25DD8B4CCEF1EF03A
:103D8000AF3DEFEF1EF0B03DEFEF1EF0B13DEFEFB6
:103D90001EF0B23DEFEF1EF02A3CEFEF1EF02B3C81
:103DA000EFEF1EF0C253D8A4DBEF1EF0C151140890
:103DB000D8B0EFEF1EF0140EC15D0101186F000EB8
:103DC0000001C2590101196F000119C11BF118C18D
:103DD0001AF10BEF1EF0010E016EF1EF1EF0000E56
:103DE000016EADEF3FF03D5001011F5DD8B003D033
:103DF00000010CEF1FF00001D8A408EF1FF0010133
:103E00001E513C5CD8A003D000010CEF1FF0000154
:103E1000000E016E1BEF1FF01FC171F11EC170F18A
:103E200049EC09F01FC13FF01EC13EF0416A41C09C
:103E300040F0010E016E000C0101216B226B236B1F
:103E4000000130EC08F001016A6B2A0E6B6F000173
:103E500009EC0BF00152D8A432EF1FF04052D8B455
:103E600088EF1FF040C020F1010120512225246F6E
:103E7000000E2321256F1F51255DD8B003D000010E
:103E80005BEF1FF00001D8A44FEF1FF001011E519E
:103E9000245DD8B003D000015BEF1FF00001010EDC
:103EA0000101216F22511E5D006E23511F59036EC7
:103EB0000050206F0001416A01012051415CD8A0EF
:103EC00003D0000174EF1FF00001420E4124E96E9F
:103ED000EA6AD8B0EA2AEFCF24F124C16EF182EC6D
:103EE00008F0412A5CEF1FF0010120513E26000E30
:103EF0003F2220512227000E23232153D8A403D090
:103F0000000186EF1FF0000188EF1FF023EF1FF084
:103F10006E50705CD8A09AEF1FF0D8A495EF1FF0F8
:103F20006F506D5CD8B09AEF1FF070C003F06F5007
:103F30009DEF1FF06EC003F06D506D6E03C06EF00C
:103F400001012251016E2351026E0001000C2990E3
:103F50002B6A2BC02AF0140EC15D01011E6F000EEA
:103F60000001C25901011F6F040E1E5D1C6F000E7F
:103F70001F591D6F19500001AF5DD8A42EEF20F01E
:103F80001A50B05DD8A42EEF20F01B50B15DD8A41C
:103F90002EEF20F01C50B25DD8A42EEF20F0080EBA
:103FA0000101556F00019DEC1BF00152D8B42EEFBA
:103FB00020F00101556B00019DEC1BF00152D8B4BB
:103FC0002EEF20F0010E01011F6F180E1E6F000171
:103FD000B9EC1BF00152D8B42EEF20F03FC01BF11A
:103FE0003EC01AF11DC11FF11CC11EF145EC1CF0B1
:103FF0001BC11FF11AC11EF1F3EC1EF02A3C2EEF7B
:1040000020F02B3C2EEF20F012EC16F00101216B7A
:10401000206B0001D0EC15F0080E01011927195191
:104020000708D8B003D000011CEF20F00001010107
:10403000182BD8B4192B000119C121F118C120F196
:10404000D0EC15F01DC11FF11CC11EF11CEC1FF0BE
:10405000CFEC16F0010E016E30EF20F0000E016E75
:10406000B6EF3FF03E503C5C006E3F503D58036E53
:104070000050016E0350026EBDEF22F001011F538C
:10408000D8A403D000016BEF20F00001010E010164
:10409000686F200E676F000197EC0BF00152D8B4E7
:1040A0006BEF20F01EC103F001011D51E96E00010C
:1040B00003C0EAFF01012051EF5CD8B403D0000136
:1040C0006BEF20F0000101011D2BD8B41E2B1F0740
:1040D00000013EEF20F001011F53D8B403D00001CE
:1040E00077EF20F00001010E016E79EF20F0000E55
:1040F000016EC2EF20F001011C6B298A020E556F80
:1041000000019DEC1BF00152D8B44AEF22F0F8EC0C
:104110001DF00152D8B44AEF22F0060E0101556F8E
:1041200000019DEC1BF00152D8B44AEF22F00101CE
:104130001F6B0D0E1E6F000145EC1CF00152D8B430
:104140004AEF22F0010E01011E6F110E1D6F0001DA
:10415000F6EC1BF00152D8B44AEF22F001011F6BBC
:10416000080E1E6F000145EC1CF00152D8B44AEF56
:1041700022F001011E6B320E1D6F060E1F6F000133
:104180003EEF20F00152D8B44AEF22F001011F6B3C
:10419000CA0E1E6F000145EC1CF00152D8B44AEF64
:1041A00022F0299829942986630E0101556F000198
:1041B0009DEC1BF00152D8B44AEF22F0820E0101AF
:1041C000556F00019DEC1BF00152D8B44AEF22F06C
:1041D000530E0101556F00019DEC1BF00152D8B444
:1041E0004AEF22F0630E0101556F00019DEC1BF0B8
:1041F0000152D8B44AEF22F0010E0101686F1A0E85
:10420000676F000197EC0BF00152D8B4A8EF21F0D2
:1042100001011A3D02D004D00001000113EF21F08A
:104220000001A8EF21F0010E0101686F1B0E676FFE
:10423000000197EC0BF00152D8B4A8EF21F0010176
:104240001A513508D8B403D000013BEF21F000012A
:1042500001011B2D02D004D0000100013BEF21F031
:104260000001010E0101686F1C0E676F000197ECE1
:104270000BF0A6EF21F001011A513308D8B403D096
:10428000000157EF21F0000101011B510408D8B4CF
:1042900003D0000157EF21F00001010E01011E6F54
:1042A0000D0E1D6F0001F6EC1BF0A6EF21F00101D1
:1042B0001A2D02D004D0000100017BEF21F0000193
:1042C00001011B510408D8B403D000017BEF21F099
:1042D000000101011C510508D8B403D000017BEF97
:1042E00021F0000101011E6B210E1D6F0001F6EC93
:1042F0001BF0A6EF21F001011A510308D8B403D036
:1043000000019FEF21F0000101011B510308D8A01B
:1043100003D000019FEF21F0000101011C510508AD
:10432000D8B403D000019FEF21F0000101011E6B02
:10433000250E1D6F0001F6EC1BF0A6EF21F0010128
:104340001F6B00011BC11EF145EC1CF0FCEF20F0BF
:10435000EC2DDAEF21F001011C510208D8B403D092
:104360000001DAEF21F00001010EEA6E030EE96EA2
:10437000E26AA60EE16E060E016EE6CFEEFF012E9A
:10438000BDEF21F0B6C00CF1B5C00BF1B4C00AF11D
:10439000B3C009F114C1FEF013C1FDF012C1FCF06D
:1043A00011C1FBF0F4C0F2F0F3C0F1F0030EEC6FBA
:1043B0004AEF22F0EC510308D8B4E4EF21F0EC51BD
:1043C0001308D8A44AEF22F001011C510508D8B403
:1043D00003D000014AEF22F00001A80EF86FC00ED2
:1043E000F76F01011053D8B403D000011AEF22F087
:1043F000000101010F53D8B403D000011AEF22F0DD
:10440000000101010E51A808D8B003D000011AEF35
:1044100022F00001D8A416EF22F001010D51BF08CF
:10442000D8B003D000011AEF22F000010EC1F8F05D
:104430000DC1F7F0F853D8A426EF22F0F7513B084E
:10444000D8A026EF22F0F86B3C0EF76FD890F83129
:10445000FA6FF731F96FF66BF56BFEC01CF0FDC01B
:104460001BF0FCC01AF0FBC019F01CEC13F064EC5C
:1044700013F0ACEC13F02EEC14F00D0E9EA83EEFF2
:1044800022F0AD6E0A0E9EA843EF22F0AD6E300E04
:10449000EC6F148E41EF23F02B6A2BC02AF0299E7B
:1044A000299001011F6BB90E1E6F0001B9EC1BF0C2
:1044B0000152D8B445EF23F001011F6BB70E1E6FF8
:1044C0000001B9EC1BF00152D8B445EF23F0010113
:1044D0001F6BE80E1E6F0001B9EC1BF00152D8B43F
:1044E00045EF23F001011F6BEA0E1E6F0001B9ECCE
:1044F0001BF00152D8B445EF23F0E953D8A486EF5E
:1045000022F0E8510708D8B045EF23F0E95105083B
:10451000D8A045EF23F0D8A493EF22F0E851C008CB
:10452000D8A045EF23F0EA51EB11D8B4CDEF22F03B
:10453000E9C022F1E8C021F170EC16F00101216B15
:10454000AF0E206F0001DBEC15F00101216BB30E03
:10455000206F0001DBEC15F001016F6B00015BECDB
:1045600008F0110E01016F6F00015BEC08F03FC015
:1045700019F13EC018F132EF20F002C01BF101C06A
:104580001AF11BC11FF11AC11EF145EC1CF019C133
:104590001FF118C11EF1F3EC1EF0EA53D8A4D5EFB9
:1045A00022F0EB53D8B4DBEF22F02A3C45EF23F0A6
:1045B0002B3C45EF23F001011D6B000183EC1BF048
:1045C0002B6A2BC02AF02990B7510708D8A408EF0E
:1045D00023F0B853D8A408EF23F00101216B1C0E7F
:1045E000206F00013CEC15F0080EE85D01011A6F28
:1045F000000E0001E95901011B6F00011BC11FF1F1
:104600001AC11EF11CEC1FF034EC17F041EF23F03F
:10461000B7510D08D8A436EF23F0B853D8A436EF1D
:1046200023F02996299429880101216B1C0E206F03
:1046300000013CEC15F001011A6B000101011A5157
:10464000000130EC00F001011A2B6D6F0001AEEC9F
:1046500008F00C0E01011A5DD8B403D000011EEF62
:1046600023F0000134EC17F041EF23F0B751440878
:10467000D8A441EF23F0B853D8A441EF23F07BEF47
:1046800020F0010E016E47EF23F0000E016EBFEF28
:104690003FF001011F51E96E2051EA6E2151EF24D4
:1046A000016E2251EC20036EE9060150EF6E00010D
:1046B00003C0ECFFE90601011F51E96E2051EA6ECB
:1046C0000001ECCF24F1ED52EFCF23F10101245191
:1046D000225DD8B003D000018BEF23F00001D8A4F5
:1046E0007BEF23F001012151235DD8A003D000010D
:1046F0008BEF23F00001020E01011F25E96E000E71
:104700002021EA6E010EEE26D8B003D000018BEF17
:1047100023F0EF2A0001000C948804009486040022
:104720008298949804008B969496A00E0101646F71
:104730000001ECEC0DF0D7C055F10101566B000102
:1047400055C164F1ECEC0DF0D6C064F1ECEC0DF069
:1047500094980000948682A6ABEF23F0040000003A
:1047600000000000948804009488040094860400EB
:104770008298949804008B969496A10E0101646F20
:104780000001ECEC0DF065EF29F00101566B576B61
:10479000586B596B5A6B5B6B5C6B5D6B5E6B5F6BE5
:1047A000606B616B626B636B646B656B666B566BA6
:1047B0000001010156510408D8B003D0000105EFF3
:1047C00024F00001010E0101686F550E676F0001B2
:1047D00097EC0BF00152D8B405EF24F001015551CC
:1047E0002008D8A003D0000105EF24F0000101014A
:1047F00055513D08D8A403D0000105EF24F0000175
:104800000101562B0001D9EF23F00101566B000185
:10481000010156510708D8B003D0000157EF24F02A
:104820000001010E0101686F550E676F000197ECE2
:104830000BF00152D8B457EF24F001015551200874
:10484000D8A003D0000157EF24F000010101555119
:104850002608D8A403D0000157EF24F00001570E1A
:1048600001015625E96E010EEA6ED8B0EA2A5551CB
:104870006008D8A003D000014EEF24F00001010130
:1048800055517A08D8B003D000014EEF24F0000152
:1048900001015551DF0B000151EF24F00101555189
:1048A0000001EF6E0101562B000108EF24F0010119
:1048B000566B0001010156510408D8B003D0000125
:1048C00086EF24F00001010E0101686F550E676F3D
:1048D000000197EC0BF00152D8B486EF24F00101EF
:1048E00055512008D8A003D0000186EF24F0000124
:1048F000010155513D08D8A403D0000186EF24F0F2
:1049000000010101562B00015AEF24F00101566B02
:104910000001010156510708D8B003D00001D8EFBB
:1049200024F00001010E0101686F550E676F000150
:1049300097EC0BF00152D8B4D8EF24F00101555197
:104940002008D8A003D00001D8EF24F00001010115
:1049500055512608D8A403D00001D8EF24F0000157
:104960005F0E01015625E96E010EEA6ED8B0EA2A03
:1049700055516008D8A003D00001CFEF24F000010A
:10498000010155517A08D8B003D00001CFEF24F0CF
:10499000000101015551DF0B0001D2EF24F00101AC
:1049A00055510001EF6E0101562B000189EF24F0F3
:1049B0000101566B0001010156510708D8B003D020
:1049C000000108EF25F00001570E01015625E96EA0
:1049D000010EEA6ED8B0EA2A0001EFCF67F15F0E50
:1049E00001015625E96E010EEA6ED8B0EA2AEF50B1
:1049F000675DD8A403D0000103EF25F00001000E8D
:104A0000016E5BEF25F00101562B0001DBEF24F076
:104A10000101566B0001010156510708D8B003D0BF
:104A2000000159EF25F000010A0E01015625676FBC
:104A3000000167C1A9FFA86AA69CA69EA684F250A1
:104A4000006EF29E0F01550EA76EAA0EA76EA682EB
:104A50000001A6B229EF25F0A6940050F2120A0E2A
:104A600001015625676F570E5625E96E010EEA6E55
:104A7000D8B0EA2A0001EFCF68F167C1A9FF68C189
:104A8000A8FFA69CA69EA684F250006EF29E0F017F
:104A9000550EA76EAA0EA76EA6820001A6B24EEF13
:104AA00025F0A6940050F2120101562B00010BEFE5
:104AB00025F0010E016EFCEF2BF00101566B576BD8
:104AC000586B596B5A6B5B6B5C6B5D6B5E6B566BBB
:104AD0000001010156510408D8B003D0000195EF40
:104AE00025F00001010E0101686F550E676F00018E
:104AF00097EC0BF00152D8B495EF25F00101555118
:104B00002008D8A003D0000195EF25F00001010195
:104B100055513D08D8A403D0000195EF25F00001C0
:104B20000101562B000169EF25F00101566B0001D0
:104B3000010156510708D8B003D00001E7EF25F076
:104B40000001010E0101686F550E676F000197ECBF
:104B50000BF00152D8B4E7EF25F0010155512008C0
:104B6000D8A003D00001E7EF25F000010101555165
:104B70003D08D8A403D00001E7EF25F00001570E4F
:104B800001015625E96E010EEA6ED8B0EA2A5551A8
:104B90006008D8A003D00001DEEF25F0000101017C
:104BA00055517A08D8B003D00001DEEF25F000019E
:104BB00001015551DF0B0001E1EF25F001015551D5
:104BC0000001EF6E0101562B000198EF25F0010165
:104BD00057513008D8B403D0000133EF26F000015C
:104BE000010158513508D8B403D0000133EF26F045
:104BF0000001010159513408D8B403D0000133EF4A
:104C000026F0000101015A513008D8B403D0000148
:104C100033EF26F0000101015B513808D8B403D00E
:104C2000000133EF26F0000101015C513608D8B4D1
:104C300003D0000133EF26F0000101015D5135087A
:104C4000D8B403D0000133EF26F0000101015E511A
:104C50003208D8B403D0000133EF26F00001010E72
:104C6000016E8BEF26F00101566B000101015651D8
:104C70000708D8B003D0000189EF26F00001570ED5
:104C800001015625E96E010EEA6ED8B0EA2AEF500E
:104C90002008D8B403D0000162EF26F000010A0E0C
:104CA00001015625606F000160C1A9FFA69CA69E68
:104CB000A680A850000AD8A462EF26F0010E016E6B
:104CC0008BEF26F0570E01015625E96E010EEA6EB4
:104CD000D8B0EA2A0001EFCF5FF10A0E0101562594
:104CE000606F000160C1A9FFA69CA69EA680A85087
:104CF00001015F5DD8A403D0000184EF26F000011C
:104D0000000E016E8BEF26F00101562B000136EFED
:104D100026F0010E016E3EEF2CF001015E516003A2
:104D20000001F3CF01F0F4CF00F001016103F35073
:104D300000265F516003F3500020026E000137EF40
:104D400027F00101586B596B5A6B5B6B5C6B5D6BA9
:104D50005B6B5A6B000101015B53D8B403D00001B7
:104D6000E1EF26F0000101015A510408D8B003D048
:104D70000001E1EF26F00001010E0101686F570EFE
:104D8000676F000197EC0BF00152D8B4E1EF26F009
:104D9000010157512008D8A003D00001E1EF26F00F
:104DA0000001010157513D08D8A403D00001E1EFF3
:104DB00026F0000101015A2BD8B45B2B0001ABEFA8
:104DC00026F001015B6B5A6B000101015B53D8B403
:104DD00003D000014AEF27F0000101015A510408F5
:104DE000D8B003D000014AEF27F00001010E010105
:104DF000686F570E676F000197EC0BF00152D8B443
:104E00004AEF27F0010157512008D8A003D0000134
:104E10004AEF27F00001010157512608D8A403D01A
:104E200000014AEF27F00001010157512F08D8A0D7
:104E300003D0000143EF27F0000101015751390869
:104E4000D8B003D0000143EF27F00001300E01017C
:104E5000575D5C6F5D6B000159C15FF158C15EF138
:104E60000101616B0A0E606F00018DEF26F002C038
:104E70005FF101C05EF101015C515E25586F5D512B
:104E80005F21596F000101015A2BD8B45B2B00013F
:104E9000E5EF26F001015851016E5951026E0001F3
:104EA000000C0F0E0101581758510908D8B003D053
:104EB000000167EF27F00001300E01015825596FFE
:104EC000000159C16DF1AEEC08F070EF27F0370E1C
:104ED00001015825596F000159C16DF1AEEC08F080
:104EE000000C01015639576F0F0E5717000157C1BB
:104EF00058F151EC27F056C158F151EC27F0000C55
:104F000055C1A9FFA69CA69EA680A8500008D8B0AF
:104F10009FEF27F055C1A9FFA69CA69EA680A8508A
:104F20000408D8A09FEF27F055C1A9FFA69CA69E14
:104F3000A680A850030F0101576F586B000155C19F
:104F4000A9FFA69CA69EA680A8500408D8B0BEEFD4
:104F500027F055C1A9FFA69CA69EA680A8500608CA
:104F6000D8A0BEEF27F055C1A9FFA69CA69EA6809B
:104F7000A850FC0F0101576F586B000155C1A9FFE4
:104F8000A69CA69EA680A8500708D8A4D3EF27F019
:104F900055C1A9FFA69CA69EA680A850010F01019D
:104FA000576F586B000155C1A9FFA69CA69EA6800D
:104FB000A8500808D8A4E8EF27F055C1A9FFA69C7F
:104FC000A69EA680A850FB0F0101576F586B0001E9
:104FD00001015751016E5851026E0001000C55C17C
:104FE000A9FFA69CA69EA680A8500108D8B403EFEE
:104FF00028F055C1A9FFA69CA69EA680A850080827
:10500000D8A409EF28F0290E016E000E026E57EFAA
:1050100028F055C1A9FFA69CA69EA680A85002080C
:10502000D8B41DEF28F055C1A9FFA69CA69EA68066
:10503000A8500308D8A423EF28F02A0E016E000E12
:10504000026E57EF28F055C1A9FFA69CA69EA68028
:10505000A8500408D8B437EF28F055C1A9FFA69C82
:10506000A69EA680A8500708D8A43DEF28F02B0ED6
:10507000016E000E026E57EF28F055C1A9FFA69CE5
:10508000A69EA680A8500508D8B451EF28F055C1B7
:10509000A9FFA69CA69EA680A8500608D8A457EFF4
:1050A00028F0280E016E000E026E57EF28F0000C5B
:1050B000006A16EC0EF094980000948682A65EEFCB
:1050C00028F004000000000000009488040005EFB0
:1050D0003AF0010E0101356F010E366F010E376F88
:1050E000386B010E396F010E3A6F010E3B6F010EE6
:1050F0003C6F010E3D6F3E6B010E3F6F010E406F26
:10510000416B010E426F010E436F446B010E456F00
:10511000010E466F476B010E486F010E496F4A6BD7
:10512000010E4B6F010E4C6F4D6B010E4E6F010E59
:105130004F6F506B010E516F010E526F536B010E8A
:10514000546F2B6A00012BC02AF02A52D8A4ACEF6E
:1051500028F02990ADEF28F02980298A470E010117
:10516000556F00019DEC1BF00152D8B409EF3AF0E5
:10517000450E0101556F00019DEC1BF00152D8B4A2
:1051800009EF3AF0540E0101556F00019DEC1BF040
:105190000152D8B409EF3AF0200E0101556F000119
:1051A0009DEC1BF02F0E0101556F00019DEC1BF0D3
:1051B00001011D6B000101011D510B08D8B003D086
:1051C000000117EF29F00001010E0101686F210EA7
:1051D000676F000197EC0BF00152D8B417EF29F07C
:1051E000010121512008D8A003D0000117EF29F0B8
:1051F0000001010121513F08D8A403D0000117EF9D
:1052000029F00001070E01011D25016E036AD8B0C7
:10521000032A0150D40FE96E000E0320EA6E00014C
:1052200021C1EFFF01011D2B0001DBEF28F001017F
:105230001D510B08D8B003D0000134EF29F0000154
:10524000070E01011D25016E036AD8B0032A015023
:10525000D40FE96E000E0320EA6EEF6A000101012F
:105260001D2B000117EF29F045EC0EF00152D8B4C8
:105270003CEF29F03FEF29F0DB6B45EC0EF02B6A99
:105280002BC02AF02990706A280E6F6EE753D8A4BD
:1052900063EF29F00101556B000101015551000137
:1052A0004FEC00F00101552B6D6F0001AEEC08F0E2
:1052B0001F0E0101555DD8B403D000014DEF29F058
:1052C000000105EF3AF08CEF23F0D451D511D8B49A
:1052D00003EF3AF0010E006E16EC0EF001C01FF164
:1052E000D451D8B4D507D407DA51010B000AD8B489
:1052F000FDEF39F001011F514008D8B403D000017F
:10530000FDEF39F00001D451D511D8B4FDEF39F0DB
:10531000010E006E16EC0EF001C01FF1D451D8B48E
:10532000D507D407300E01011F5D206F1F514008C3
:10533000D8A003D00001A3EF29F00001370E01012E
:105340001F5D206F00010101202D02D004D000015B
:10535000000192EF2BF00001010E0101556F0001D9
:1053600013EC0DF003C02CF102C02BF101C02AF1A7
:1053700000C029F101011D6B000101011D511F0831
:10538000D8B003D000010BEF2AF000012CC130F19E
:105390002BC12FF12AC12EF129C12DF1350E0101AA
:1053A0001D25E96E010EEA6ED8B0EA2A000130C16F
:1053B0005BF12FC15AF12EC159F12DC158F10101F4
:1053C0001D51576FD8A403D00001F6EF29F000015A
:1053D000D89001015B335A3359335833572F02D0D9
:1053E00004D000010001E8EF29F00001010158514B
:1053F000010B006E5951000B016E5A51000B026EE9
:105400005B51000B036E000100C0EFFF01011D2B7B
:105410000001BDEF29F0030E01011D6F0001010124
:105420001D510608D8B003D0000190EF2AF000010A
:1054300001011D51040DF350350FE96E010EEA6EA6
:10544000D8B0EA2AEF52D8A403D000012CEF2AF0FA
:105450000001310E2DEF2AF0300E0101576F0001CF
:1054600057C16EF182EC08F001011D51040DF3509B
:10547000010F350FE96E010EEA6ED8B0EA2AEF523D
:10548000D8A403D0000149EF2AF00001310E4AEF01
:105490002AF0300E0101576F000157C16EF182EC06
:1054A00008F001011D51040DF350020F350FE96E94
:1054B000010EEA6ED8B0EA2AEF52D8A403D0000158
:1054C00066EF2AF00001310E67EF2AF0300E01017D
:1054D000576F000157C16EF182EC08F001011D51B8
:1054E000040DF350030F350FE96E010EEA6ED8B0CC
:1054F000EA2AEF52D8A403D0000183EF2AF000017A
:10550000310E84EF2AF0300E0101576F000157C1B0
:105510006EF182EC08F001011D2B00010FEF2AF063
:10552000000E81BA010E000AD8A41BEF2BF0010176
:105530001D6B000101011D510108D8B003D000010D
:105540001BEF2BF0000101011D51040DF350350F2D
:10555000E96E010EEA6ED8B0EA2AEF52D8A403D061
:105560000001B7EF2AF00001310EB8EF2AF0300E3B
:105570000101576F000157C16EF182EC08F0010183
:105580001D51040DF350010F350FE96E010EEA6E47
:10559000D8B0EA2AEF52D8A403D00001D4EF2AF001
:1055A0000001310ED5EF2AF0300E0101576F0001D6
:1055B00057C16EF182EC08F001011D51040DF3504A
:1055C000020F350FE96E010EEA6ED8B0EA2AEF52EB
:1055D000D8A403D00001F1EF2AF00001310EF2EF60
:1055E0002AF0300E0101576F000157C16EF182ECB5
:1055F00008F001011D51040DF350030F350FE96E42
:10560000010EEA6ED8B0EA2AEF52D8A403D0000106
:105610000EEF2BF00001310E0FEF2BF0300E0101D9
:10562000576F000157C16EF182EC08F001011D2B8C
:1056300000019AEF2AF0070E01011D6F1D51040DA4
:10564000F350350FE96E010EEA6ED8B0EA2AEF5238
:10565000D8A403D0000131EF2BF00001310E32EF5E
:105660002BF0300E0101576F000157C16EF182EC33
:1056700008F001011D51040DF350010F350FE96EC3
:10568000010EEA6ED8B0EA2AEF52D8A403D0000186
:105690004EEF2BF00001310E4FEF2BF0300E0101D9
:1056A000576F000157C16EF182EC08F001011D51E6
:1056B000040DF350020F350FE96E010EEA6ED8B0FB
:1056C000EA2AEF52D8A403D000016BEF2BF00001BF
:1056D000310E6CEF2BF0300E0101576F000157C1F6
:1056E0006EF182EC08F001011D51040DF350030F1F
:1056F000350FE96E010EEA6ED8B0EA2AEF52D8A44F
:1057000003D0000188EF2BF00001310E89EF2BF060
:10571000300E0101576F000157C16EF182EC08F0A5
:10572000FBEF39F0010120510208D8B403D0000189
:10573000BBEF2BF00001080EA96EA69CA69EA680CA
:10574000A850000AD8A4B9EF2BF00101556B000155
:1057500001015551000167EC00F00009D8B4B9EF20
:105760002BF00101552B6E6F000182EC08F0A8EFC1
:105770002BF0FBEF39F0010120510308D8B403D01E
:105780000001E4EF2BF00001080EA96EA69CA69E76
:10579000A680A8500108D8A4E2EF2BF00101556BB8
:1057A000000101015551000167EC00F00009D8B477
:1057B000E2EF2BF00101552B6E6F000182EC08F037
:1057C000D1EF2BF0FBEF39F0010120510408D8B4E0
:1057D00003D00001F1EF2BF00001010E156EFBEF7D
:1057E00039F0010120510608D8B403D0000133EF8D
:1057F0002CF00001C5EF23F001C01DF101011D2DAA
:1058000002D004D0000100011DEF2CF000010101C5
:10581000556B000101015551000173EC00F00009C6
:10582000D8B41BEF2CF00101552B6E6F000182ECF8
:1058300008F00AEF2CF031EF2CF00101556B00015C
:1058400001015551000182EC00F00009D8B431EF9C
:105850002CF00101552B6E6F000182EC08F020EF57
:105860002CF0FBEF39F0010120510708D8B403D028
:10587000000155EF2CF000015DEF25F001C01DF196
:1058800001011D53D8A403D000014BEF2CF00001FF
:10589000310E4CEF2CF0300E0101556F000155C157
:1058A0006EF182EC08F0FBEF39F00101205108089D
:1058B000D8B403D00001BCEF2CF000010101646BEF
:1058C00000011CC063F1C8EC12F02E0E01016E6FD6
:1058D000000182EC08F00101646B00011BC063F160
:1058E000C8EC12F02E0E01016E6F000182EC08F080
:1058F0000101646B00011AC063F1C8EC12F02E0EB6
:1059000001016E6F000182EC08F00101646B00017F
:1059100019C063F1C8EC12F01752D8A4A6EF2CF00E
:105920000101556B00010101555100018FEC00F0A0
:105930000009D8B4A4EF2CF00101552B6E6F0001C3
:1059400082EC08F093EF2CF0BAEF2CF00101556BCC
:1059500000010101555100019BEC00F00009D8B491
:10596000BAEF2CF00101552B6E6F000182EC08F0AC
:10597000A9EF2CF0FBEF39F0010120510908D8B450
:1059800003D000016BEF2EF00001A96A36C0A8FF1A
:10599000A69CA69EA684F250006EF29E0F01550EA4
:1059A000A76EAA0EA76EA6820001A6B2D5EF2CF0B4
:1059B000A6940050F212010EA96E37C0A8FFA69C53
:1059C000A69EA684F250006EF29E0F01550EA76EA1
:1059D000AA0EA76EA6820001A6B2ECEF2CF0A69448
:1059E0000050F212A1EC26F002C056F101C055F1B0
:1059F000020EA96E55C1A8FFA69CA69EA684F250D1
:105A0000006EF29E0F01550EA76EAA0EA76EA6821B
:105A10000001A6B209EF2DF0A6940050F212A1ECFD
:105A200026F002C056F101C055F1030EA96E55C112
:105A3000A8FFA69CA69EA684F250006EF29E0F01BF
:105A4000550EA76EAA0EA76EA6820001A6B226EF7B
:105A50002DF0A6940050F212A1EC26F002C056F1EF
:105A600001C055F1040EA96E55C1A8FFA69CA69EC3
:105A7000A684F250006EF29E0F01550EA76EAA0E7C
:105A8000A76EA6820001A6B243EF2DF0A6940050A7
:105A9000F212A1EC26F002C056F101C055F1050E3C
:105AA000A96E55C1A8FFA69CA69EA684F250006EC2
:105AB000F29E0F01550EA76EAA0EA76EA6820001D8
:105AC000A6B260EF2DF0A6940050F212A1EC26F0E1
:105AD00002C056F101C055F1130EA96E55C1A8FFC1
:105AE000A69CA69EA684F250006EF29E0F01550E53
:105AF000A76EAA0EA76EA6820001A6B27DEF2DF0BA
:105B0000A6940050F212A1EC26F002C056F101C09A
:105B100055F1140EA96E55C1A8FFA69CA69EA68499
:105B2000F250006EF29E0F01550EA76EAA0EA76EE0
:105B3000A6820001A6B29AEF2DF0A6940050F212B0
:105B4000A1EC26F002C056F101C055F1150EA96E68
:105B500055C1A8FFA69CA69EA684F250006EF29E98
:105B60000F01550EA76EAA0EA76EA6820001A6B25F
:105B7000B7EF2DF0A6940050F212A1EC26F002C06F
:105B800056F101C055F1160EA96E55C1A8FFA69C8D
:105B9000A69EA684F250006EF29E0F01550EA76ECF
:105BA000AA0EA76EA6820001A6B2D4EF2DF0A6948D
:105BB0000050F212A1EC26F002C056F101C055F1DE
:105BC000170EA96E55C1A8FFA69CA69EA684F250EA
:105BD000006EF29E0F01550EA76EAA0EA76EA6824A
:105BE0000001A6B2F1EF2DF0A6940050F212A1EC44
:105BF00026F002C056F101C055F1180EA96E55C12C
:105C0000A8FFA69CA69EA684F250006EF29E0F01ED
:105C1000550EA76EAA0EA76EA6820001A6B20EEFC1
:105C20002EF0A6940050F212A1EC26F002C056F11C
:105C300001C055F1190EA96E55C1A8FFA69CA69EDC
:105C4000A684F250006EF29E0F01550EA76EAA0EAA
:105C5000A76EA6820001A6B22BEF2EF0A6940050EC
:105C6000F212A1EC26F002C056F101C055F11A0E55
:105C7000A96E55C1A8FFA69CA69EA684F250006EF0
:105C8000F29E0F01550EA76EAA0EA76EA682000106
:105C9000A6B248EF2EF0A6940050F21212EC02F0D9
:105CA00001C055F1060EA96E55C1A8FFA69CA69E7F
:105CB000A684F250006EF29E0F01550EA76EAA0E3A
:105CC000A76EA6820001A6B263EF2EF0A694005044
:105CD000F212FBEF39F0010120510A08D8B403D0C9
:105CE0000001F7EF2FF00001010E926E90EC03F02F
:105CF000040E01011E6F000101011E510708D8B0FA
:105D000003D0000133EF2FF000011EC157F189ECE1
:105D10000DF001012C6B2B6B000102C02AF101C0B8
:105D200029F101011D6B000101011D511F08D8B0AF
:105D300003D00001E2EF2EF000012CC130F12BC1A5
:105D40002FF12AC12EF129C12DF1350E01011D259A
:105D5000E96E010EEA6ED8B0EA2A000130C15BF1AB
:105D60002FC15AF12EC159F12DC158F101011D5118
:105D7000576FD8A403D00001CDEF2EF00001D890CA
:105D800001015B335A3359335833572F02D004D0B3
:105D900000010001BFEF2EF0000101015851010B7D
:105DA000006E5951000B016E5A51000B026E5B518F
:105DB000000B036E000100C0EFFF01011D2B00016D
:105DC00094EF2EF001013653D8A403D00001EDEF7B
:105DD0002EF00001310EEEEF2EF0300E0101556F66
:105DE000000155C16EF182EC08F001013753D8A4CF
:105DF00003D0000100EF2FF00001310E01EF2FF072
:105E0000300E0101556F000155C16EF182EC08F0B2
:105E100001013853D8A403D0000113EF2FF0000183
:105E2000310E14EF2FF0300E0101556F000155C1F6
:105E30006EF182EC08F001013D53D8A403D00001BB
:105E400026EF2FF00001310E27EF2FF0300E010169
:105E5000556F000155C16EF182EC08F001011E2B57
:105E600000017CEF2EF0000E81BA010E000AD8A4CA
:105E7000F5EF2FF0010E01011E6F000101011E510F
:105E80000208D8B003D00001F5EF2FF000011EC1C9
:105E900057F189EC0DF001012C6B2B6B000102C056
:105EA0002AF101C029F101011D6B000101011D5101
:105EB0001F08D8B003D00001A4EF2FF000012CC1BF
:105EC00030F12BC12FF12AC12EF129C12DF1350E50
:105ED00001011D25E96E010EEA6ED8B0EA2A000123
:105EE00030C15BF12FC15AF12EC159F12DC158F1CA
:105EF00001011D51576FD8A403D000018FEF2FF07F
:105F00000001D89001015B335A3359335833572F6E
:105F100002D004D00001000181EF2FF00001010147
:105F20005851010B006E5951000B016E5A51000B74
:105F3000026E5B51000B036E000100C0EFFF010118
:105F40001D2B000156EF2FF001013653D8A403D0CA
:105F50000001AFEF2FF00001310EB0EF2FF0300E47
:105F60000101556F000155C16EF182EC08F001018D
:105F70003753D8A403D00001C2EF2FF00001310E37
:105F8000C3EF2FF0300E0101556F000155C16EF1C6
:105F900082EC08F001013853D8A403D00001D5EFFA
:105FA0002FF00001310ED6EF2FF0300E0101556FAA
:105FB000000155C16EF182EC08F001013D53D8A4F7
:105FC00003D00001E8EF2FF00001310EE9EF2FF0D0
:105FD000300E0101556F000155C16EF182EC08F0E1
:105FE00001011E2B00013EEF2FF0FBEF39F0010104
:105FF00020510C08D8B403D0000118EF30F0000194
:10600000060EA96EA86AA69CA69EA684F250006EF3
:10601000F29E0F01550EA76EAA0EA76EA682000172
:10602000A6B210EF30F0A6940050F212FBEF39F058
:10603000010120510D08D8B403D0000136EF31F032
:106040000001010E926E01011D6B000101011D5145
:106050001208D8B003D0000149EF30F00001350E2E
:1060600001011D25016E010E036ED8B0032A0150F7
:10607000556F000103C056F1A1EC26F056C1EAFFAE
:1060800055C1E9FF01C0EFFF01011D2B000126EF03
:1060900030F0040E01011E6F000101011E510708BE
:1060A000D8B003D00001BBEF30F000011EC157F1A2
:1060B00089EC0DF002C026F101C025F10101255146
:1060C000F00B556F2651566F1E51030DF350F60F0E
:1060D000350FE96E010EEA6ED8B0EA2AEF50080DCE
:1060E000F35055255A6F000E56215B6F1E51030D5C
:1060F000F350F50F350FE96E010EEA6ED8B0EA2ABB
:10610000EF50040DF3505A255F6F000E5B21606F56
:106110001E51030DF350F40F350FE96E010EEA6EB8
:10612000D8B0EA2AD890EF34006E5F25646F000E75
:106130006021656F2551010B006E2651000B036E27
:1061400000506425276F03506521286F000190ECF3
:1061500003F028C155F10101566B00011EC15CF12D
:1061600055C15DF127C15EF1E6EC03F001011E2B84
:1061700000014DEF30F0000E81BA010E000AD8A4E4
:1061800034EF31F0010E01011E6F000101011E51BB
:106190000208D8B003D0000134EF31F000011EC175
:1061A00057F189EC0DF002C026F101C025F1010183
:1061B0002551F00B556F2651566F1E51030DF350AC
:1061C0000B0F350FE96E010EEA6ED8B0EA2AEF50D8
:1061D000080DF35055255A6F000E56215B6F1E5166
:1061E000030DF3500A0F350FE96E010EEA6ED8B0B9
:1061F000EA2AEF50040DF3505A255F6F000E5B2121
:10620000606F1E51030DF350090F350FE96E010E3B
:10621000EA6ED8B0EA2AD890EF34006E5F25646F3A
:10622000000E6021656F2551010B006E2651000B99
:10623000036E00506425276F03506521286F00010D
:1062400090EC03F028C155F10101566B00011EC10D
:106250005CF155C15DF127C15EF1E6EC03F001018F
:106260001E2B0001C6EF30F0FBEF39F00101205189
:106270000E08D8B403D00001CBEF31F00001010EBD
:10628000926E90EC03F0A1EC26F002C056F101C032
:1062900055F1080EA96E55C1A8FFA69CA69EA6841E
:1062A000F250006EF29E0F01550EA76EAA0EA76E59
:1062B000A6820001A6B25AEF31F0A6940050F21265
:1062C000080EA96EA69CA69EA680A8500108D8A478
:1062D00076EF31F0110E01015C6FFF0E5D6F200E45
:1062E0005E6F0001E6EC03F0C9EF31F0110E010121
:1062F0005C6FFF0E5D6F5E6B0001E6EC03F0010E5C
:10630000926E90EC03F0010E01011E6F000101017D
:106310001E510708D8B003D00001C9EF31F00001C9
:106320001EC157F189EC0DF001012C6B2B6B0001A4
:1063300002C02AF101C029F101012951E00B256FAA
:106340002A51266F29510F0B276F2A51000B286FF6
:1063500027512525296F285126212A6F2B6B2C6B5D
:10636000000190EC03F02AC156F12BC157F12CC16A
:1063700058F10101596B00011EC15CF156C15DF17C
:1063800029C15EF1E6EC03F001011E2B000187EF4D
:1063900031F0FBEF39F0010120510F08D8B403D0E0
:1063A0000001EEEF31F00001A9EC05F0120EA96E2C
:1063B000A86AA69CA69EA684F250006EF29E0F01CB
:1063C000550EA76EAA0EA76EA6820001A6B2E6EF32
:1063D00031F0A6940050F212FBEF39F00101205188
:1063E0001008D8B403D0000107EF32F00001090E05
:1063F000A96EA69CA69EA680A8500101556F646B4D
:10640000000155C163F1C8EC12F0FBEF39F0010156
:1064100020511108D8B403D000012FEF32F0000151
:10642000A1EC26F002C056F101C055F1090EA96E8B
:1064300055C1A8FFA69CA69EA684F250006EF29EAF
:106440000F01550EA76EAA0EA76EA6820001A6B276
:1064500027EF32F0A6940050F212FBEF39F0010161
:1064600020511208D8B403D0000158EF32F00001D7
:10647000120EA96EA69CA69EA680A850000AD8A4BB
:1064800056EF32F00101556B000101015551000139
:1064900067EC00F00009D8B456EF32F00101552B3B
:1064A0006E6F000182EC08F045EF32F0FBEF39F03F
:1064B000010120511308D8B403D0000181EF32F05C
:1064C0000001120EA96EA69CA69EA680A8500108E7
:1064D000D8A47FEF32F00101556B00010101555145
:1064E000000167EC00F00009D8B47FEF32F0010141
:1064F000552B6E6F000182EC08F06EEF32F0FBEF6F
:1065000039F0010120511408D8B403D00001A9EFDB
:1065100032F00001A1EC26F002C056F101C055F1A5
:10652000120EA96E55C1A8FFA69CA69EA684F25085
:10653000006EF29E0F01550EA76EAA0EA76EA682E0
:106540000001A6B2A1EF32F0A6940050F212FBEFC8
:1065500039F0010120511508D8B403D000018EEFA5
:1065600033F00001010E926E090EA96EA69CA69E44
:10657000A680A850120F0101566F000156C157F1B5
:1065800089EC0DF001012C6B2B6B000102C02AF18C
:1065900001C029F101011D6B000101011D510F080E
:1065A000D8B003D000011BEF33F000012CC130F153
:1065B0002BC12FF12AC12EF129C12DF1350E010178
:1065C0001D25E96E010EEA6ED8B0EA2A000130C13D
:1065D0005BF12FC15AF12EC159F12DC158F10101C2
:1065E0001D51576FD8A403D0000106EF33F000010E
:1065F000D89001015B335A3359335833572F02D0A7
:1066000004D000010001F8EF32F0000101015851FF
:10661000010B006E5951000B016E5A51000B026EB6
:106620005B51000B036E000100C0EFFF01011D2B49
:106630000001CDEF32F0030E01011D6F00010101D9
:106640001D510608D8B003D0000147EF33F0000118
:10665000350E01011D25E96E010EEA6ED8B0EA2A59
:10666000EF52D8A403D000013AEF33F00001310E0D
:106670003BEF33F0300E0101556F000155C16EF153
:1066800082EC08F001011D2B00011FEF33F0000E1A
:1066900081BA010E000AD8A479EF33F001011D6B15
:1066A000000101011D510108D8B003D0000179EFAC
:1066B00033F00001350E01011D25E96E010EEA6E71
:1066C000D8B0EA2AEF52D8A403D000016CEF33F01F
:1066D0000001310E6DEF33F0300E0101556F0001F6
:1066E00055C16EF182EC08F001011D2B000151EF44
:1066F00033F001013C53D8A403D0000184EF33F000
:106700000001310E85EF33F0300E0101556F0001AD
:1067100055C16EF182EC08F0FBEF39F00101205118
:106720001608D8B403D00001C2EF33F00001010114
:106730001D6B000101011D510408D8B003D00001F8
:10674000BCEF33F00001320E01011D25E96EEA6A4B
:10675000D8B0EA2A0001EFCF55F155C156F171ECDE
:1067600027F03A0E01016E6F000182EC08F0010182
:106770001D2B00019AEF33F037C056F171EC27F072
:10678000FBEF39F0010120511B08D8B403D0000100
:10679000EAEF33F00001A1EC26F002C026F101C0BF
:1067A00025F1A1EC26F002C028F101C027F1010E6D
:1067B000926E90EC03F028C155F10101566B000177
:1067C00025C15CF155C15DF127C15EF1E6EC03F036
:1067D000FBEF39F0010120511C08D8B403D00001AF
:1067E00023EF34F000010101646B000124C063F168
:1067F000C8EC12F02E0E01016E6F000182EC08F061
:106800000101646B000123C063F1C8EC12F02E0E8D
:1068100001016E6F000182EC08F00101646B000160
:1068200022C063F1C8EC12F02E0E01016E6F000160
:1068300082EC08F00101646B000121C063F1C8EC37
:1068400012F0FBEF39F0010120511D08D8B403D03C
:1068500000015CEF34F000010101646B000128C00D
:1068600063F1C8EC12F02E0E01016E6F000182EC94
:1068700008F00101646B000127C063F1C8EC12F05D
:106880002E0E01016E6F000182EC08F00101646BB5
:10689000000126C063F1C8EC12F02E0E01016E6FEC
:1068A000000182EC08F00101646B000125C063F176
:1068B000C8EC12F0FBEF39F0010120511E08D8B4EA
:1068C00003D000010EEF35F00001010E926E0101C0
:1068D000286B276B030E1D6F000101011D51060877
:1068E000D8B003D000019AEF34F00001A1EC26F0FB
:1068F00002C026F101C025F126C103F00101255196
:10690000026E1D51006ED8A403D000018FEF34F049
:106910000001D89002360336002E89EF34F0025081
:106920000101272703502823000101011D2B00012D
:106930006DEF34F0000E81BA010E000AD8A4D1EF39
:1069400034F001011D6B000101011D510108D8B097
:1069500003D00001D1EF34F00001A1EC26F002C019
:1069600026F101C025F126C103F001012551026E77
:106970001D51006ED8A403D00001C6EF34F0000111
:10698000D89002360336002EC0EF34F002500101D9
:10699000272703502823000101011D2B0001A4EF2C
:1069A00034F0A1EC26F002C026F101C025F101016E
:1069B0002535026E2635036E02360336023603365F
:1069C0000236033602360336023603360236033603
:1069D000800E02160250272703502823040E272773
:1069E000FF0E2823000190EC03F0090EA96EA69C6F
:1069F000A69EA680A850120F0101566F000128C163
:106A000057F10101586B000156C15CF157C15DF1AE
:106A100027C15EF1E6EC03F0FBEF39F001012051F4
:106A20002008D8B403D000012DEF35F0000101019A
:106A3000556B0001010155510001A8EC00F000095F
:106A4000D8B42BEF35F00101552B6E6F000182ECAD
:106A500008F01AEF35F0FBEF39F001012051210861
:106A6000D8B403D000014CEF35F000010101556BA3
:106A70000001010155510001BAEC00F00009D8B441
:106A80004AEF35F00101552B6E6F000182EC08F0E2
:106A900039EF35F0FBEF39F0010120512208D8B46D
:106AA00003D0000188EF35F00001000E81BA010E1D
:106AB000000AD8A472EF35F00101556B0001010105
:106AC00055510001C7EC00F00009D8B470EF35F063
:106AD0000101552B6E6F000182EC08F05FEF35F07D
:106AE00086EF35F00101556B0001010155510001A0
:106AF000D5EC00F00009D8B486EF35F00101552B34
:106B00006E6F000182EC08F075EF35F0FBEF39F0A5
:106B1000010120512308D8B403D00001A7EF35F0BC
:106B200000010101556B0001010155510001E3EC29
:106B300000F00009D8B4A5EF35F00101552B6E6FB8
:106B4000000182EC08F094EF35F0FBEF39F0010121
:106B500020512A08D8B403D00001C0EF35F000015D
:106B6000020EA96EA69CA69EA680A8500101556F94
:106B7000646B000155C163F1C8EC12F0FBEF39F012
:106B8000010120512B08D8B403D00001D9EF35F012
:106B90000001030EA96EA69CA69EA680A850010126
:106BA000556F646B000155C163F1C8EC12F0FBEF47
:106BB00039F0010120512C08D8B403D00001F2EFC4
:106BC00035F00001040EA96EA69CA69EA680A850D2
:106BD0000101556F646B000155C163F1C8EC12F0FF
:106BE000FBEF39F0010120512D08D8B403D000018A
:106BF0000BEF36F00001050EA96EA69CA69EA6809E
:106C0000A8500101556F646B000155C163F1C8ECD8
:106C100012F0FBEF39F0010120512E08D8B403D057
:106C2000000124EF36F00001130EA96EA69CA69E6B
:106C3000A680A8500101556F646B000155C163F136
:106C4000C8EC12F0FBEF39F0010120512F08D8B445
:106C500003D000013DEF36F00001140EA96EA69C92
:106C6000A69EA680A8500101556F646B000155C116
:106C700063F1C8EC12F0FBEF39F00101205130084C
:106C8000D8B403D0000156EF36F00001150EA96EFE
:106C9000A69CA69EA680A8500101556F646B0001BA
:106CA00055C163F1C8EC12F0FBEF39F0010120513E
:106CB0003108D8B403D000016FEF36F00001160E92
:106CC000A96EA69CA69EA680A8500101556F646B74
:106CD000000155C163F1C8EC12F0FBEF39F001017E
:106CE00020513208D8B403D0000188EF36F00001FB
:106CF000170EA96EA69CA69EA680A8500101556FEE
:106D0000646B000155C163F1C8EC12F0FBEF39F080
:106D1000010120513308D8B403D00001A1EF36F0AF
:106D20000001180EA96EA69CA69EA680A85001017F
:106D3000556F646B000155C163F1C8EC12F0FBEFB5
:106D400039F0010120513408D8B403D00001BAEF62
:106D500036F00001190EA96EA69CA69EA680A8502A
:106D60000101556F646B000155C163F1C8EC12F06D
:106D7000FBEF39F0010120513508D8B403D00001F0
:106D8000D3EF36F000011A0EA96EA69CA69EA6802F
:106D9000A8500101556F646B000155C163F1C8EC47
:106DA00012F0FBEF39F0010120513608D8B403D0BE
:106DB0000001E7EF37F00001010E926E90EC03F056
:106DC0000101566B1B0E556F000180EC27F002C0CD
:106DD00056F101C055F155C157F189EC0DF0010193
:106DE0002C6B2B6B000102C02AF101C029F10A0EA5
:106DF00001011D6F000101011D510D08D8B003D024
:106E0000000149EF37F000012CC130F12BC12FF107
:106E10002AC12EF129C12DF1350E01011D25E96E82
:106E2000010EEA6ED8B0EA2A000130C15BF12FC131
:106E30005AF12EC159F12DC158F101011D51576F61
:106E4000D8A403D0000134EF37F00001D89001013D
:106E50005B335A3359335833572F02D004D00001D3
:106E6000000126EF37F0000101015851010B006EBF
:106E70005951000B016E5A51000B026E5B51000B11
:106E8000036E000100C0EFFF01011D2B0001FBEFAD
:106E900036F00101566B1B0E556F0001EFEC27F029
:106EA00002C056F101C055F155C157F189EC0DF002
:106EB00001012C6B2B6B000102C02AF101C029F1EA
:106EC0001B0EA96EA69CA69EA680A8500108D8B449
:106ED00088EF37F01B0EA96EA69CA69EA680A85030
:106EE0000308D8B488EF37F01B0EA96EA69CA69EA7
:106EF000A680A8500608D8B488EF37F01B0EA96EFC
:106F0000A69CA69EA680A8500708D8A493EF37F0A9
:106F10002AC129F12BC12AF12CC12BF101012C6BC3
:106F200000019BEF37F0000E01012A17000E2B170E
:106F3000000E2C170001010129372A372B372C3777
:106F400029372A372B372C3729372A372B372C3735
:106F500029372A372B372C37F00E29174251080DC5
:106F6000F3502925556F000E2A21566F000E2B2154
:106F7000576F000E2C21586F4151040DF3505525C9
:106F8000596F000E56215A6F000E57215B6F000E8D
:106F900058215C6FD8904035006E59255D6F000E0A
:106FA0005A215E6F000E5B215F6F000E5C21606FE7
:106FB0003F515D25616F000E5E21626F000162C16D
:106FC00064F161C163F1C8EC12F0FBEF39F001012B
:106FD00020513708D8B403D0000100EF38F0000189
:106FE0001B0EA96EA69CA69EA680A8500101556FF7
:106FF000646B000155C163F1C8EC12F0FBEF39F08E
:10700000010120513808D8B403D0000128EF38F02E
:107010000001A1EC26F002C056F101C055F11B0E93
:10702000A96E55C1A8FFA69CA69EA684F250006E2C
:10703000F29E0F01550EA76EAA0EA76EA682000142
:10704000A6B220EF38F0A6940050F212FBEF39F010
:10705000010120513908D8B403D000016BEF39F099
:107060000001010E926EA1EC26F001C041F11B0E51
:10707000A96EA69CA69EA680A8500808D8B44BEF7F
:1070800038F0080EA96EA69CA69EA680A850000AFD
:10709000D8A44EEF38F00101416B0001A1EC26F0BD
:1070A00002C026F101C025F101012653D8B403D056
:1070B000000165EF38F00001010125510008D8A05A
:1070C00003D0000169EF39F00001010126510F08DA
:1070D000D8B003D0000169EF39F0000126C128F1D2
:1070E00025C127F1010127510F0B556F2851000BC6
:1070F000566F276B5535286F2837FC0E2817566BAF
:107100001B0E556F000180EC27F002C056F101C044
:1071100055F155C157F189EC0DF001012C6B2B6B2A
:10712000000102C02AF101C029F101012999C30E11
:107130002A17000E2B17000E2C1727512925556FE3
:1071400028512A21566F000E2B21576F000E2C213B
:10715000586F4139006EF00E001600505525296F0A
:10716000000E56212A6F000E57212B6F000E58215A
:107170002C6F000190EC03F00101566B1B0E556F54
:10718000000180EC27F002C056F101C055F12AC180
:1071900058F12BC159F12CC15AF101015B6B00016F
:1071A00055C15CF158C15DF129C15EF1E6EC03F017
:1071B00026C128F125C127F10101283327332833BF
:1071C000273328332733283327330F0E28171B0E76
:1071D000A96EA69CA69EA680A8500108D8A403D09C
:1071E000000112EF39F000011B0EA96EA69CA69EAD
:1071F000A680A8500308D8B412EF39F01B0EA96E70
:10720000A69CA69EA680A8500608D8B412EF39F016
:107210001B0EA96EA69CA69EA680A8500708D8A4FF
:107220003CEF39F00101566B1B0E556F0001EFEC7E
:1072300027F002C056F101C055F155C157F189EC54
:107240000DF002C026F101C025F190EC03F0010120
:10725000566B1B0E556F0001EFEC27F002C056F184
:1072600001C055F155C15CF127C15DF125C15EF149
:10727000E6EC03F069EF39F00101566B1B0E556F18
:107280000001EFEC27F002C056F101C055F155C1E5
:1072900057F189EC0DF002C026F101C025F190EC08
:1072A00003F00101566B1B0E556F0001EFEC27F048
:1072B00002C056F101C055F126C157F10101586BCA
:1072C000000155C15CF157C15DF127C15EF1E6ECEB
:1072D00003F0FBEF39F0010120513A08D8B403D094
:1072E0000001F5EF39F00001010E926E90EC03F011
:1072F0000101566B1B0E556F000180EC27F002C098
:1073000056F101C055F155C157F189EC0DF001015D
:107310002C6B2B6B000102C02AF101C029F1010185
:107320001D6B000101011D510F08D8B003D00001F1
:10733000E0EF39F000012CC130F12BC12FF12AC14F
:107340002EF129C12DF1350E01011D25E96E010E29
:10735000EA6ED8B0EA2A000130C15BF12FC15AF1C0
:107360002EC159F12DC158F101011D51576FD8A4FB
:1073700003D00001CBEF39F00001D89001015B335D
:107380005A3359335833572F02D004D0000100012B
:10739000BDEF39F0000101015851010B006E595148
:1073A000000B016E5A51000B026E5B51000B036E15
:1073B000000100C0EFFF01011D2B000192EF39F029
:1073C00001013953D8A403D00001EBEF39F00001DB
:1073D000310EECEF39F0300E0101556F000155C14F
:1073E0006EF182EC08F0FBEF39F03F0E01016E6F99
:1073F000000182EC08F001EF3AF01FC16EF182EC5F
:1074000008F065EF29F058EF28F0010E016E0BEF40
:107410003AF0000E016EC3EF3CF0080EAD6FAC6B9E
:107420002990C3C02AF0C4C02BF0B8C021F1B7C066
:1074300020F1D0EC15F0BAC021F1B9C020F1D0ECA8
:1074400015F00101216BCA0E206F000165EC15F0EB
:107450000101216BC60E206F000165EC15F00101E2
:107460001E51020B000AD8A403D000013CEF3AF0F1
:107470000001600E3DEF3AF0500E01011F6F000158
:107480001FC16EF182EC08F01EC16EF182EC08F0B3
:107490000B0E01016E6F000182EC08F0B80E0101C5
:1074A0006E6F000182EC08F001011E51020B000A10
:1074B000D8A403D0000180EF3AF000010101216B54
:1074C000280E206F00013CEC15F0020E01016E6FDA
:1074D000000182EC08F0040E01016E6F000182ECE5
:1074E00008F0050E0101216FB40E206F0001D0ECF1
:1074F00015F00101216B240E206F00013CEC15F00A
:107500000101216B190E206F0001DBEC15F0010168
:10751000216BB30E206F0001DBEC15F001016F6BE6
:1075200000015BEC08F0060E01016F6F00015BECDF
:1075300008F0140EC15D01011F6F000E0001C25959
:107540000101206F000120C122F11FC121F170EC67
:1075500016F02A5001011F6F1F1F00011FC16EF19D
:1075600082EC08F02B5001011F6F1F1F00011FC18B
:107570006EF182EC08F00101216B206B0001D0EC70
:1075800015F001011E51020B000AD8A403D000011E
:10759000D2EF3AF000010101216B2C0E206F0001A7
:1075A0003CEC15F006EF3BF030EC08F02AC0C3F0DD
:1075B0002BC0C4F06E52D8A4E6EF3AF06D50270805
:1075C000D8A0E6EF3AF06E6A280E6D6E01011D51EB
:1075D000020B000AD8A403D00001F4EF3AF0000136
:1075E000040E6D26000E6E226EC0C2F06DC0C1F09A
:1075F0000101216B206B00013CEC15F0060EAE6F13
:1076000012EC16F01DC11EF10DEF3AF0CFEC16F0A2
:10761000D3EF3CF0100E01011A6F29902B6A000184
:107620002BC02AF001011F6BB90E1E6F0001B9ECCF
:107630001BF00152D8B4D7EF3CF001011F6BB70E1D
:107640001E6F0001B9EC1BF00152D8B4D7EF3CF02B
:1076500001011E6BC60E1D6F0001F6EC1BF00152FE
:10766000D8B4D7EF3CF001011E6BCA0E1D6F0001AC
:10767000F6EC1BF00152D8B4D7EF3CF0010E01013B
:10768000686F180E676F000197EC0BF00152D8B4C9
:10769000D7EF3CF0010E0101686F190E676F000112
:1076A00097EC0BF00152D8B4D7EF3CF001011F6BFF
:1076B000060E1E6F000145EC1CF00152D8B4D7EF46
:1076C0003CF0C253D8A46AEF3BF0C1512708D8B0B0
:1076D000D7EF3CF01950AF5DD8A4D7EF3CF01A506B
:1076E000B05DD8A4D7EF3CF01B50B15DD8A4D7EF64
:1076F0003CF01C50B25DD8A4D7EF3CF0140EC15D35
:1077000001011D6F000E0001C25901011E6F000131
:107710001EC122F11DC121F170EC16F00101216B97
:10772000190E206F0001DBEC15F00101216BB30E87
:10773000206F0001DBEC15F001016F6B00015BECC9
:1077400008F0060E01016F6F00015BEC08F001010B
:1077500018515008D8A003D00001CDEF3BF0000134
:10776000C153D8A4B8EF3BF0C253D8B4CDEF3BF02F
:1077700001011F6B040E1E6F000145EC1CF001524D
:10778000D8B4CDEF3BF0040EC15F000EC25B100E0B
:107790000101185F0001A7EF3BF0280EC15DD06F1B
:1077A000000EC259D16F3FC01CF13EC01BF1D1C0C9
:1077B0001FF1D0C01EF145EC1CF01CC11FF11BC114
:1077C0001EF1F3EC1EF02A3CD7EF3CF02B3CD7EF38
:1077D0003CF001011D6B000183EC1BF00101216BEA
:1077E000280E206F00013CEC15F0C46BC4C0C3F040
:1077F00029962994298801011951040B000AD8A45B
:1078000003D000010AEF3CF0000101011A6B0001F6
:10781000C7EF3CF001011951020B000AD8A403D0B4
:10782000000149EF3CF000010101206BC60E1F6F03
:10783000226B010E216F000149EC23F0B7510D08B6
:10784000D8A427EF3CF0B853D8B430EF3CF0B75190
:107850005008D8A443EF3CF0B853D8A443EF3CF011
:10786000FF0ECB6FFF0ECA6FCF51036ECE51CE2BE2
:10787000D8B4CF2BCC6F03C0CDF0120E01011A6F1C
:10788000000147EF3CF0140E01011A6F0001C7EF31
:107890003CF001011951010B000AD8A403D00001EA
:1078A00068EF3CF00001010ED02501011D6F000EB4
:1078B0000001D12101011E6F206BC60E1F6F000158
:1078C0001EC122F11DC121F149EC23F0C7EF3CF0AC
:1078D00001011951100B000AD8A403D00001C7EF11
:1078E0003CF00001D051D111D8B484EF3CF001013B
:1078F000206BC60E1F6F0001D1C022F1D0C021F154
:1079000049EC23F087EF3CF001011A6B0001B751FD
:107910000D08D8A4B3EF3CF0B853D8A4B3EF3CF0B3
:10792000CA53D8A4B3EF3CF0CB53D8A4B3EF3CF088
:1079300001011D6B000101011D51000130EC00F03F
:1079400001011D2B6D6F0001AEEC08F00C0E010162
:107950001D5DD8B403D000019BEF3CF0110E1A6FEF
:107960000001C7EF3CF0B7515008D8A4C7EF3CF076
:10797000B853D8A4C7EF3CF0D051D111D8B4C7EF59
:107980003CF069EF28F0110E01011A6F00010101AE
:107990001A53D8A403D00001D3EF3CF000011AC160
:1079A0001DF1D4EF3AF0010E016ED9EF3CF0000E5C
:1079B000016EC8EF3FF0F86AD08EFE0E006E050E25
:1079C000016EEA6A020EE96EEF6AE92AD8B4EA2A81
:1079D000002EE4EF3CF0012EE4EF3CF0EA6AE96AA5
:1079E000070EC16E056A066A010E076E086A096A0B
:1079F0000A6A0B6A810EAF6E260EAC6E900EAB6EED
:107A0000156A166A060E186E326A400E336EF60E4E
:107A1000346EFD0E356E366A376AC56BEC6B01014C
:107A2000156B166B0001F29CF29EF2BE14EF3DF056
:107A3000130E926E826AFF0E946EFF0E956E848016
:107A400084828484969096929694000E80B8010E5B
:107A5000000AD8A499EF3DF0140E0101186F00013F
:107A6000FA0E0101646F0001D5EC01F00101182F3D
:107A700002D003D000010001F3D7000E80B8010E40
:107A8000000AD8B403D0000199EF3DF00001A96AC3
:107A9000A69CA69EA680A850366E010EA96EA69C36
:107AA000A69EA680A850376E01011B6B190E1A6F97
:107AB000C00E1C6FA80E1D6F1E6B020E1F6F000103
:107AC000EBEC01F001011B6B210E1A6FFF0E1C6F16
:107AD000FF0E1D6FFF0E1E6F1F6B0001EBEC01F020
:107AE00001011B6B250E1A6FC00E1C6FA80E1D6FB7
:107AF0001E6B010E1F6F0001EBEC01F033EC02F086
:107B0000120EA96E010EA86EA69CA69EA684F25027
:107B1000006EF29E0F01550EA76EAA0EA76EA682EA
:107B20000001A6B291EF3DF0A6940050F212A9EC2C
:107B300005F0F19ECF6AB50ECD6ECD9E0101216B91
:107B4000120E206F236B226B000145EC07F01486A8
:107B5000149A149880848086298629842998FE0E98
:107B6000946E8B808B901E0E0101646F0001D5EC2A
:107B700001F0640E0101646F0001D5EC01F08B800F
:107B80001E0E0101646F0001D5EC01F0FF0E946E32
:107B90000101186B00010101185100011CEC01F0FA
:107BA0000101182B00019EA8D3EF3DF0AD6E040E2D
:107BB0000101185DD8B403D00001CBEF3DF0000EF9
:107BC00081BA010E000AD8B403D0000103EF3EF0E1
:107BD00000010101186B0001010118510001C7ECFF
:107BE00000F00101182B00019EA8F4EF3DF0AD6EEE
:107BF0000A0E0101185DD8B403D00001ECEF3DF08E
:107C000000011BEF3EF00101186B0001010118514A
:107C10000001D5EC00F00101182B00019EA80EEF29
:107C20003EF0AD6E0A0E0101185DD8B403D000011C
:107C300006EF3EF00001200E01016D6F0001AEEC79
:107C400008F00101186B000101011851000127EC37
:107C500001F00101182B6D6F0001AEEC08F00F0E62
:107C60000101185DD8B403D0000124EF3EF0030EEB
:107C7000196F0001390E01016D6F0001AEEC08F0C3
:107C80000101192F02D004D0000100013AEF3EF0AB
:107C9000200E6D6F0001AEEC08F00101186B0001C1
:107CA000010118510001BAEC00F00101182B6D6FB1
:107CB0000001AEEC08F0080E0101185DD8B403D045
:107CC000000150EF3EF00A0E6D6F0001AEEC08F0BF
:107CD000CEEC08F00152D8A4D0EF3EF00101186BB1
:107CE000000101011851000137EC01F00101182BCE
:107CF0006D6F0001AEEC08F0070E0101185DD8B4FD
:107D000003D0000171EF3EF00001A5EF0CF00A0E68
:107D1000A96E310EA86EA69CA69EA684F250006E97
:107D2000F29E0F01550EA76EAA0EA76EA682000145
:107D3000A6B298EF3EF0A6940050F2120B0EA96E78
:107D4000320EA86EA69CA69EA684F250006EF29EED
:107D50000F01550EA76EAA0EA76EA6820001A6B24D
:107D6000AFEF3EF0A6940050F2120C0EA96E330E47
:107D7000A86EA69CA69EA684F250006EF29E0F01ED
:107D8000550EA76EAA0EA76EA6820001A6B2C6EF78
:107D90003EF0A6940050F212A9EC05F068EF3EF018
:107DA0002DEF0FF059EC11F0120EA96EA69CA69EB5
:107DB000A680A850176E1752D8A4E5EF3EF01C6AB3
:107DC0001B6A1A6A196AF0EF3EF0148ECEEC08F0C6
:107DD0001CEC13F064EC13F0ACEC13F02EEC14F08C
:107DE0000D0E9EA8F1EF3EF0AD6E0A0E9EA8F6EFC6
:107DF0003EF0AD6E090EA96E020EA86EA69CA69E60
:107E0000A684F250006EF29E0F01550EA76EAA0EC8
:107E1000A76EA6820001A6B20BEF3FF0A694005019
:107E2000F2121B0EA96E010EA86EA69CA69EA68439
:107E3000F250006EF29E0F01550EA76EAA0EA76EAD
:107E4000A6820001A6B222EF3FF0A6940050F212E3
:107E5000000E80B8010E000AD8A468EF3FF00D0EA6
:107E60009EA830EF3FF0AD6E0A0E9EA835EF3FF0B2
:107E7000AD6E0101176B0001010117513F08D8B029
:107E800003D0000167EF3FF0000117C157F189EC03
:107E90000DF002C019F101C018F119C11FF1370E20
:107EA0000101206F0001F4EC13F018C11FF1370E2F
:107EB0000101206F0001F4EC13F0200E9EA85EEF8C
:107EC0003FF0AD6E0101172B00013CEF3FF08088C1
:107ED000BCEC09F01752D8A475EF3FF01850165CAF
:107EE000D8B075EF3FF017EF19F01752D8A48BEF09
:107EF0003FF01850165CD8A08BEF3FF0148ECEECFC
:107F000008F01CEC13F064EC13F0ACEC13F02EEC66
:107F100014F0010E176E85EF1AF00152D8B4CAEFB3
:107F20003FF001011D6B000183EC1BF0AC51060812
:107F3000D8A4A2EF3FF0AD510808D8A4A2EF3FF0BB
:107F40002EEF1DF0AC53D8A4C8EF3FF0AD51080898
:107F5000D8A4C8EF3FF044EF1EF00152D8B4C8EFE8
:107F60003FF0AE2DB8EF3FF0A7EF1FF0C8EF3FF0A6
:107F7000AE511108D8A4C1EF3FF04CEF22F0C8EF8A
:107F80003FF0AE510608D8A4C8EF3FF00AEF3BF02F
:107F90003D6A3C6A152CCEEF3FF0FF0028EF3FF022
:027FA0000300DC
:020000040030CA
:0C000000FFFAFCFEFFFFFBFFFFFFFFFF0D
:00000001FF
